:020000040000FA
:06400000A5EF21F0120003
:06400800EAEF31F01200A6
:06402A00080058410000EF
:1040300062000000030000005B410000A7000000D8
:104040001600000071410000670100006C000000D4
:10405000DD410000000E0000310000000E420000B3
:10406000000100006700000075420000000400002D
:10407000BF000000344300006000000001000000A9
:0C4080003543000061000000010000005A
:044158000000010062
:05415B000A0D41737321
:104160006572743A20002C206C696E6520000A0D7F
:01417000004E
:0F4171000F0F02030100140000002F00000000D8
:104180005761726E696E673A2077726F6E67206F43
:1041900072206E6F20666F726D6174004C464E2007
:1041A000656E7472790064656C2066696C65000ADE
:1041B0000D436172642070726573656E74000A0D40
:1041C0004361726420676F6E650066696C652E637B
:0D41D00000444154412020202020202000E8
:0341DD004C4F47FD
:1041E00046494C45312E4353560044656D6F6E73FE
:1041F00074726174696F6E2052756E6E696E6700BD
:0F420000000000000000000100000001010100AB
:02420E000A0D97
:104210004346444C2044656D6F2056657220302E15
:1042200030410A0D000A0D5573652068656C7020D9
:10423000746F207072696E7420636F6D6D616E644F
:104240002064657461696C73000A0D5373736D6D3E
:104250006868777764646D6D79793C63723E202D70
:104260002057726974652054696D6520616E642001
:06427000446174650000CA
:0B427500426F6F74207265636F72640B
:1042800020736563746F723A200042797465207000
:10429000657220736563746F723A200053656374AE
:1042A0006F72732070657220636C75737465723AF7
:1042B0002000436F70696573207065722046415419
:1042C0003A20004D617820726F6F7420656E7472B1
:1042D0006965733A2000536563746F72732070656B
:1042E00072204641543A2000526F6F742073656308
:1042F000746F723A20004D61782064697220736592
:1043000063746F72733A2000446174612073656353
:10431000746F723A200046415420312073656374F3
:104320006F723A2000464154203220736563746FE7
:05433000723A200000BC
:02433400000087
:02433500000086
:0A4336008680120086901200867047
:0A43400012008650010B00D012009D
:06434A001DEE00F02DEE57
:1043500000F0F86A189C78EC22F074EC30F0FDD78D
:02436000120049
:0E4362000C6A0B6A100EE76ED8900F361036FC
:104370000B360C3614500B5C15500C5805E31450DA
:0E4380000B5E15500C5A0F2AE72EF0D71200D4
:02438E000C6AB7
:104390000B6A0A6A180EE76ED8900E360F36103682
:1043A0000A360B360C3613500A5C14500B58155055
:1043B0000C5807E313500A5E14500B5A15500C5A50
:0843C0000E2AE72EEAD71200D5
:0843C8000C6A0B6A0A6A096A1B
:1043D000200EE76ED8900D360E360F3610360936A1
:1043E0000A360B360C361250095C13500A5814501A
:1043F0000B5815500C5809E31250095E13500A5A15
:1044000014500B5A15500C5A0D2AE72EE4D71200FF
:10441000F26AF168C00EF06E9E6AA16AA46A9D6A93
:10442000A06AA36A9F6AA26AA56AD08ECD6ACF6A83
:10443000CE6ABA6ABC6ABB6AC26A090EC16EC06A39
:10444000070EB46EB56AAC6AAB6AAF6A6C6A6B6A27
:104450006F6A806A2F0E926E816AFD0E936E826A79
:10446000930E946E836A9568E70E846E180E966EAE
:10447000100E856E090E976E040E866E986E1200F1
:104480000D501202F3CF09F0F4CF0AF01302F350EB
:104490000A26000EF4200B6E0D501402F3500B266A
:1044A000000EF4200C6E0D501502F3500C260E5029
:1044B0001202F3500A26F4500B22000E0C220E506A
:1044C0001302F3500B26F4500C220E501402F3503A
:1044D0000C260F501202F3500B26F4500C220F50F2
:1044E0001302F3500C2610501202F3500C26120047
:1044F0002A0EF66E400EF76E000EF86E00010900EF
:10450000F5506A6F0900F5506B6F03E16A6701D0DF
:104510003DD00900F550656F0900F550666F090040
:10452000F550676F09000900F550E96E0900F55074
:10453000EA6E090009000900F550686F0900F5509E
:10454000696F09000900F6CF6CF0F7CF6DF0F8CF76
:104550006EF065C0F6FF66C0F7FF67C0F8FF0001A8
:10456000685302E1695307E00900F550EE6E6807F1
:10457000F8E26907F9D76CC0F6FF6DC0F7FF6EC0AF
:0E458000F8FF00016A07000E6B5BBFD7120048
:02458E00D9CF83
:10459000E6FFE1CFD9FFFD0EDBCFE6FFFE0EDBCF5E
:1045A000E6FFCCEC27F0E552E552BA0EE66E000EBF
:1045B000E66ECCEC27F0E552E552E552E7CFD9FFA5
:1045C0001200D9CFE6FFE1CFD9FF070EE126D9507F
:1045D000FD0FE96EFF0EDA20EA6EEE50ED103AE0C4
:1045E000A70EE66E000EE66ECCEC27F0E552E55223
:1045F000FB0EDBCFE6FFFC0EDBCFE6FFCCEC27F0BB
:10460000E552E552B20EE66E000EE66ECCEC27F0F7
:10461000E552E552D9CFE6FFDACFE6FFF90EDBCF60
:10462000E6FFFA0EDBCFE6FF94EC26F0E106E106AA
:10463000E106E106D9CFE6FFDACFE6FFCCEC27F0C2
:10464000E552E552BA0EE66E000EE66ECCEC27F0AF
:10465000E552E552D9CFE1FFE552E7CFD9FF12008D
:10466000000EE66E010EE66ECCEC27F0E552E55248
:1046700000017F6B806B1200D9CFE6FFE1CFD9FF3D
:10468000050EE126D9CFE6FFDACFE6FFAEEC24F047
:10469000E552E55200095CE0000EDF9E0D0EDF5C86
:1046A00047E100017F51EA6A6F0FE96E000EEA22CE
:1046B000EF6A610E6F5D04E36F517A0801E36F9B4F
:1046C0006F0EE66E000EE66E17EC28F0E552E5522E
:1046D00000016F51470A26E0140A1BE01B0A08E09C
:1046E000770A06E0740A01E020D0F2EC3FF01DD01A
:1046F000170EE66E010EE66ECCEC27F0E552E552A1
:104700003B0EE66E010EE66ECCEC27F0E552E5526C
:104710000CD0700EE66E000EE66E31EC39F0E5520C
:10472000E55203D0A8EC3CF000D000017F6B10D024
:104730000A0EDF5C0DE00F0E00017F5D09E27F5184
:10474000EA6A6F0FE96E000EEA22DFCFEFFF7F2BE0
:0C475000D9CFE1FFE552E7CFD9FF1200FE
:04475C00D9CFE6FFCC
:10476000E1CFD9FFFD0EDB5014E1FE0EDB50030A52
:104770000DE0010A09E0030A05E0010A01E008D0A2
:10478000939406D0939604D0939802D0939A00D035
:1047900013D0FE0EDB50030A0DE0010A09E0030A04
:1047A00005E0010A01E008D0938406D0938604D086
:1047B000938802D0938A00D0E552E7CFD9FF120048
:1047C000D9CFE6FFE1CFD9FFFD0EDB5014E1FE0E9D
:1047D000DB50030A0DE0010A09E0030A05E0010AC3
:1047E00001E008D0819406D0819604D0819802D04F
:1047F000819A00D013D0FE0EDB50030A0DE0010AAF
:1048000009E0030A05E0010A01E008D0818406D02E
:10481000818604D0818802D0818A00D0E552E7CF1A
:10482000D9FF1200D9CFE6FFE1CFD9FFFE0EDB5052
:10483000030A0DE0010A09E0030A05E0010A01E0AC
:1048400008D0817406D0817604D0817802D0817A34
:1048500000D0E552E7CFD9FF1200D9CFE6FFE1CF74
:10486000D9FFE652DF6AFE0EDB50030A16E0010AAA
:104870000FE0030A08E0010A01E014D081A402D08D
:10488000010EDF6E0FD081A602D0010EDF6E0AD0BE
:1048900081A802D0010EDF6E05D081AA02D0010EE0
:1048A000DF6E00D0DF5000D0E552E552E7CFD9FFF0
:0248B0001200F4
:0E48B200D9CFE6FFE1CFD9FF0001615102E04E
:1048C000000E1AD00301416B426B436B846B856B06
:1048D000866B6C84FE0EDB506F6EA588A58AA38A5A
:1048E000858A858E6C8A6B886B8EFD0EDBCF00F31C
:1048F00000016169FF0E00D0E552E7CFD9FF120039
:104900006C6A6B6AA398A39A829C829E8594859612
:10491000859A859E0001616B1200D9CFE6FFE1CF39
:10492000D9FF0001615114E0400E0301435D10E224
:104930004151EA6A010FE96E030EEA22FE0EDBCF57
:10494000EFFF412B3F0E4117432BA388FF0E02D0F0
:10495000000E00D0E552E7CFD9FF1200D9CFE6FF15
:10496000E1CFD9FF000161511BE00301865100082E
:1049700017E28551EA6A440FE96E030EEA22EF500E
:10498000E66EFD0EDBCFE9FFFE0EDBCFEAFFE55260
:10499000E750EF6E852B3F0E85178607FF0E02D07E
:1049A000000E00D0E552E7CFD9FF1200E9CFE4FFB7
:1049B000EACFE4FFE6520301435100080DE2425101
:1049C000EA6A010FE96E030EEA22EF506D6E422B88
:1049D0003F0E4217430701D0A398E552E5CFEAFF07
:1049E000E5CFE9FF1100E9CFE4FFEACFE4FFE652AB
:1049F000400E0301865D0DE28451EA6A440FE96EC0
:104A0000030EEA226ECFEFFF842B3F0E8417862B16
:104A100002D06E50E86EE552E5CFEAFFE5CFE9FF40
:024A2000110083
:0E4A2200D9CFE6FFE1CFD9FF0001605102E0DD
:104A3000000E1CD00E01526B536B546B756B766B72
:104A4000776BAC84FE0EDB50AF6E9F889F8A9D8A89
:104A5000FD0EDBB0858C858A858EAC8AAB88AB8EEB
:104A6000DBCF31FE00016069FF0E00D0E552E7CFD9
:104A7000D9FF1200AC6AAB6A9D989D9A829C829E77
:104A800085948596859C859A859E0001606B1200B1
:104A9000D9CFE6FFE1CFD9FF0001605114E0200E2D
:104AA0000E01545D10E25251EA6A320FE96E0E0EA9
:104AB000EA22FE0EDBCFEFFF522B1F0E5217542BB4
:104AC0009D88FF0E02D0000E00D0E552E7CFD9FF3F
:104AD0001200D9CFE6FFE1CFD9FF000160511BE002
:104AE0000E017751000817E27651EA6A550FE96E18
:104AF0000E0EEA22EF50E66EFD0EDBCFE9FFFE0E52
:104B0000DBCFEAFFE552E750EF6E762B1F0E7617EC
:104B10007707FF0E02D0000E00D0E552E7CFD9FF95
:104B20001200E9CFE4FFEACFE4FFE6520E01545150
:104B300000080DE25351EA6A320FE96E0E0EEA22C6
:104B4000EF50AD6E532B1F0E5317540701D09D9895
:104B5000E552E5CFEAFFE5CFE9FF1100E9CFE4FF39
:104B6000EACFE4FFE652200E0E01775D0DE27551AB
:104B7000EA6A550FE96E0E0EEA22AECFEFFF752BF3
:104B80001F0E7517772B02D0AE50E86EE552E5CFB9
:084B9000EAFFE5CFE9FF110087
:084B9800176AE86A15AED9EFB7
:104BA00025F0126C131E141E151E1322142215223A
:104BB000171E10AEE4EF25F00D6C0E1E0F1E101E1A
:104BC0000E220F221022171EE4EC21F010BEFBEF84
:104BD00025F017AE000C0D6C0E1E0F1E101EE86A9D
:104BE0000E220F221022096C0A1E0B1E0C1E0A2216
:104BF0000B220C22000C17BEEBEF25F01888FF0CDF
:104C000010C01CF00FC01BF00F501402F4CF0EF0B8
:104C1000F3CF0DF010501502F4CF10F0F3CF0FF0DA
:104C20001402F3500E26F4500F22E86A10221B5093
:104C30001502F3500E26F4500F22E86A102215AE2A
:104C400026EF26F01B500F5E1C50105A1CAE000CB5
:104C500014500F5E1550105A000C0FC01BF00F506F
:104C60001402F4CF0EF0F3CF0DF010501502F4CF74
:104C700010F0F3CF0FF01402F3500E26F4500F2271
:104C8000E86A10221B501502F3500E26F4500F2232
:104C9000E86A1022000C10C01CF00FC01BF00EC000
:104CA0001AF00E501302F4CF0CF0F3CF0BF00F50AC
:104CB0001402F4CF0EF0F3CF0DF01302F3500C26D4
:104CC000F4500D22E86A0E221A501402F3500C26FA
:104CD000F4500D22E86A0E2210501302F3500D26F4
:104CE000F4500E22105014020F6AE86A0F22F3509B
:104CF0000E26F4500F221A501502F3500D26F450D0
:104D00000E22106AE86A0F2210221B501502F3507F
:104D10000E26F4500F22E86A10221C501502F350A0
:084D20000F26F4501022000CD4
:084D2800D9CFE6FFE1CFD9FF6E
:104D3000050EE126040EDB6A100EF36E020EF3CFB1
:104D4000DBFF270EF36E030EF3CFDBFFD950020F0C
:104D5000E96EDACFEAFFEE50ED1071E0FD0EDBCF29
:104D60000FF0FE0EDBCF10F0020EDBCF14F0030EBF
:104D7000DBCF15F0B1EC21F00FC0DEFF10C0DDFF7E
:104D8000D9CFE9FFDACFEAFFEE50ED100DE1040EC6
:104D9000DB500AE1D950020FE96EDACFEAFF010ECB
:104DA000EE1801E1ED501AE1010EF36E040EF3CF9F
:104DB000DBFFDECF00F0DDCF01F0300E0026000E6D
:104DC0000122FB0EDBCFE9FFFC0EDBCFEAFF00C0C8
:104DD000EFFFFB0EDB2AFC0E01E3DB2AFD0EDBCF2F
:104DE00002F0FE0EDBCF03F0020EDBCF0FF0030E5E
:104DF000DBCF10F0DECF14F0DDCF15F02DEC26F078
:104E00000D50025C006E0E500358016EFD0E00C086
:104E1000DBFFFE0E01C0DBFFD950020FE96EDACFD7
:104E2000EAFF0A0E146E156AEECF0FF0EDCF10F008
:104E3000B1EC21F00FC0EEFF10C0EDFF87D7FB0EE5
:104E4000DBCFE9FFFC0EDBCFEAFFEF6AD9CFE1FF52
:104E5000E552E7CFD9FF1200D9CFE6FFE1CFD9FF66
:104E6000E652DF6AFD0EDBCFE9FFFE0EDBCFEAFF85
:104E7000EF5013E00A0EDF02F3CFDFFFFD0EDBCFB2
:104E8000E9FFFE0EDBCFEAFFEF50D00FDF26FD0E6D
:104E9000DB2AFE0E01E3DB2AE5D7DF5000D0E55226
:104EA000E552E7CFD9FF1200D9CFE6FFE1CFD9FF16
:104EB000020EE126DE6ADD6AFD0EDBCFE9FFFE0EA3
:104EC000DBCFEAFFEF501EE0D9CFE9FFDACFEAFFF0
:104ED0000A0EEC02F3CFEDFFEF02F3CFEEFFF4503A
:104EE000ED26FD0EDBCFE9FFFE0EDBCFEAFFEF5034
:104EF000D00FDE26000EDD22FD0EDB2AFE0E01E3C2
:104F0000DB2ADAD7DECF00F0DDCF01F000C0F3FFFF
:104F100001C0F4FF00D0D9CFE1FFE552E7CFD9FFC0
:104F20001200D9CFE6FFE1CFD9FFFE0EDBCFE6FFBF
:104F30008DEC24F0E552000901E1F7D7E552E7CF07
:104F4000D9FF1200D9CFE6FFE1CFD9FFE652FE0E1E
:104F5000DB380F0BDF6EDF50090803E2370EDF2668
:104F600002D0300EDF26DFCFE6FFDBDFE552FE0E9C
:104F7000DB500F0BDF6EDF50090803E2370EDF2630
:104F800002D0300EDF26DFCFE6FFCBDFE552E55261
:104F9000E552E7CFD9FF1200D9CFE6FFE1CFD9FF25
:104FA000FD0EDBCFE9FFFE0EDBCFEAFFEF5010E096
:104FB000FD0EDBCFE9FFFE0EDBCFEAFFEF50E66E22
:104FC000B0DFE552FD0EDB2AFE0E01E3DB2AE8D757
:104FD000E552E7CFD9FF1200D9CFE6FFE1CFD9FFE5
:104FE000060EE126D9CFE6FFDACFE6FFFD0EDBCFD6
:104FF000E6FFFE0EDBCFE6FF97DEE106E106E10607
:10500000E106D9CFE6FFDACFE6FFC6DFE552E5528B
:10501000D9CFE1FFE552E7CFD9FF12000D0EE66EC2
:1050200080DFE5520A0EE66E7CDFE5521200D9CF32
:10503000E6FFE1CFD9FFFD0EDBCFE6FFFE0EDBCFB3
:10504000E6FFAADFE552E552E9DFE552E7CFD9FFF7
:105050001200D9CFE6FFE1CFD9FF020EE126FD0E07
:10506000DB2AFE0E01E3DB2AFD0EDBCFE9FFFE0E9D
:10507000DBCFEAFFEF50DE6EDD6AD9CFE9FFDACF92
:10508000EAFFF0CFEFFFF06AFD0EDB06FE0E01E255
:10509000DB06FD0EDBCFE9FFFE0EDBCFEAFFEF50B4
:1050A000DE26000EDD22DECF00F0DDCF01F000C0F5
:1050B000F3FF01C0F4FF00D0D9CFE1FFE552E7CF05
:1050C000D9FF1200D9CFE6FFE1CFD9FF070EE126C5
:1050D000060EDB6A100EF36E030EF3CFDBFF270E16
:1050E000F36E040EF3CFDBFF050EDB6A030EDBCF9E
:1050F00000F0040EDBCF01F0050EDBCF02F0005014
:105100000110021001E1A8D0FC0EDBCF00F0FD0E73
:10511000DBCF01F0FE0EDBCF02F000C00EF001C0CD
:105120000FF002C010F0030EDBCF13F0040EDBCF44
:1051300014F0050EDBCF15F0C7EC21F00EC0DFFF39
:10514000010E0FC0DBFF020E10C0DBFFDFCF00F04F
:10515000010EDBCF01F0020EDBCF02F00050011098
:1051600002100FE1060EDB500CE1D950030FE96E7F
:10517000DACFEAFF010EEE1803E1EE5001E1EE5046
:105180001FE1010EF36E060EF3CFDBFFDFCF00F061
:10519000010EDBCF01F0020EDBCF02F0300E002655
:1051A000000E01220222FA0EDBCFE9FFFB0EDBCF5D
:1051B000EAFF00C0EFFFFA0EDB2AFB0E01E3DB2A59
:1051C000FC0EDBCF03F0FD0EDBCF04F0FE0EDBCFD9
:1051D00005F0DFCF06F0010EDBCF07F0020EDBCFCC
:1051E00008F006C00EF007C00FF008C010F0030E64
:1051F000DBCF13F0040EDBCF14F0050EDBCF15F080
:105200004BEC26F00B50035C006E0C500458016E02
:105210000D500558026EFC0E00C0DBFFFD0E01C0F4
:10522000DBFFFE0E02C0DBFFD950030FE96EDACFC1
:10523000EAFF0A0E136E146A156AEECF0EF0EECF77
:105240000FF0EFCF10F0C7EC21F010C0EDFF0FC052
:10525000EDFF0EC0EFFF4AD7FA0EDBCFE9FFFB0EE2
:10526000DBCFEAFFEF6AD9CFE1FFE552E7CFD9FF05
:0252700012002A
:0E527200CD6ACF6ACE6ABA6ABC6ABB6AC26AEB
:10528000C16AC06A85909780809A928A8092928241
:105290008090928080969286809492840001626BC6
:1052A0001200D9CFE6FFE1CFD9FF050EE126DE6877
:1052B000010EDD6E020EDB68010EF36E030EF3CFFE
:1052C000DBFFC30EC2160C0EC212020EDBCF00F0C3
:1052D000030EDBCF01F00150000AE8AE02D001342A
:1052E00005D0030ED8800054000E015453E2D9CFEC
:1052F000E9FFDACFEAFF020EEECFDBFF030EEDCFC0
:10530000DBFF040EDB6ADB50006E016A0150000A0D
:10531000E8AE02D0D89004D0960E005C000E015882
:1053200003E2040EDB2AEFD7C282C2B2FED7C43832
:10533000F00BDE6EDD6AD9CFE9FFDACFEAFF040EAB
:10534000D890EE36ED36E806FBE1C350DE26000EBF
:10535000DD22DECF00F0DDCF01F0D950020FE96E83
:10536000DACFEAFF0050EE5E0150ED5A020EDBCFBD
:1053700000F0030EDBCF01F00001800E011509E003
:10538000D950020FE96EDACFEAFFEE6CEF1E000E85
:10539000ED229BD7DECF92F0DDCF93F00001190E06
:1053A0009303F3CF93F09203F3CF92F0F45093274B
:1053B000D9CFE1FFE552E7CFD9FF1200D9CFE6FF01
:1053C000E1CFD9FF0001625102E0000E29D0CD6A81
:1053D0000B0EBA6EFD0EDBCF00F0FE0EDBCF01F040
:1053E00001C000F0016A0050BC6EFF0EE76EFD0EBA
:1053F000DBCF00F0FE0EDBCF01F0E7500016016AB4
:105400000050BB6EC26A090EC16E810EC06EC280B2
:10541000CD806269FC0EDBCF89F043DFFF0E00D048
:10542000E552E7CFD9FF120039EF29F0D9CFE6FFD7
:10543000E1CFD9FF080EE12600016351020A30E0F6
:10544000030A2AE0010A01E044D1010E0001891596
:105450000001641504E0C30EC216140EC212020E3F
:10546000000189150001641503E0C30EC216C2884D
:10547000040E000189150001641503E0C30EC21675
:10548000C284080E000189150001641502E0C30EF4
:10549000C216010E636F1DD1C282020E636F19D155
:1054A000C2B216D1DF6A010E64C0DBFF0F0E6417B3
:1054B0006451000806E2DF2A649064430F0E64170B
:1054C000F7D7010EDB50E824646F00018951000119
:1054D000D880645502E2010E646FC438F00BE66EAA
:1054E000DF04E96EEA6AD890E936EA36810EE926E9
:1054F000000EEA22E552E750EE6EED6ADF04E96E37
:10550000EA6AD890E936EA36810EE926000EEA22E8
:10551000040ED890EE36ED36E806FBE1C350006E7F
:10552000016ADF04E96EEA6AD890E936EA36810E4C
:10553000E926000EEA220050EE260150ED22DF049B
:10554000E96EEA6AD890E936EA36810EE926000E5D
:10555000EA22020EEECFDBFF030EEDCFDBFFDF040E
:10556000E96EEA6AD890E936EA368A0EE926000E34
:10557000EA22EECF00F0EFCF01F0DF04E96EEA6A35
:10558000D890E936EA36810EE926000EEA2200506C
:10559000EE260150ED22DF04E96EEA6AD890E93682
:1055A000EA368A0EE926000EEA22020EDBCFEEFF73
:1055B000030EDBCFEDFFDF04E96EEA6AD890E9362F
:1055C000EA36810EE926000EEA22EECF00F0EFCF98
:1055D00001F0026A036A01AE02D002680368040E99
:1055E00000C0DBFF050E01C0DBFF060E02C0DBFFC3
:1055F000070E03C0DBFFD950040FE96EDACFEAFFD4
:10560000D890EF36010EEB36020EEB36030EEB367A
:10561000D950040FE96EDACFEAFFFE0EEE5E070EF8
:10562000EE5A000EEE5AEE5AD950040FE96EDACF58
:10563000EAFFE70E126E310E136E146A156AEECF92
:105640000DF0EECF0EF0EECF0FF0EFCF10F040ECFC
:1056500022F00CC0EDFF0BC0EDFF0AC0EDFF09C04A
:10566000EFFF92C000F093C001F0026A036AD950C4
:10567000040FE96EDACFEAFF00C012F001C013F0A8
:1056800002C014F003C015F0EECF0DF0EECF0EF017
:10569000EECF0FF0EFCF10F0CCEC25F010C0EDFF07
:1056A0000FC0EDFF0EC0EDFF0DC0EFFFDF04E96E90
:1056B000EA6AD890E936EA36810EE926000EEA2237
:1056C000040EDBCFEEFF050EDBCFEDFF0001636BB9
:1056D00000D0D9CFE1FFE552E7CFD9FF1200D9CFF3
:1056E000E6FFE1CFD9FF090EE126FE0EDB04E96EED
:1056F000EA6AD890E936EA36810EE926000EEA22F7
:10570000EECF00F0EFCF01F0026A036A01AE02D0E3
:105710000268036800C0DFFF010E01C0DBFF020E5C
:1057200002C0DBFF030E03C0DBFFD9CFE9FFDACFF6
:10573000EAFF020EE76ED890000EEF36010EEB3650
:10574000020EEB36030EEB36E706F5E1D9CFE9FFA3
:10575000DACFEAFFE76ED890000EEF36010EEB3697
:10576000020EEB36030EEB36E706F5E1D9CFE9FF83
:10577000DACFEAFFF40E126E010E136E146A156A88
:10578000EECF0DF0EECF0EF0EECF0FF0EFCF10F02A
:1057900040EC22F00CC0EDFF0BC0EDFF0AC0EDFFA6
:1057A00009C0EFFFD9CFE9FFDACFEAFF9A0E126EF8
:1057B000190E136E146A156AEECF0DF0EECF0EF0CF
:1057C000EECF0FF0EFCF10F0CCEC25F010C0EDFFD6
:1057D0000FC0EDFF0EC0EDFF0DC0EFFFD9CFE9FF09
:1057E000DACFEAFF030EEB50000AE8AE02D0D89001
:1057F00008D0000EEE5C000EEE58000EEE58000EC3
:10580000EE5809E3FC0EDBCFE9FFFD0EDBCFEAFF2C
:105810002B0EEF6E17D0FC0EDBCFE9FFFD0EDBCFBA
:10582000EAFF2D0EEF6ED9CFE9FFDACFEAFF000EC7
:10583000EE6CEF1EEE22EF1EEE22EF1EEF22ED5277
:10584000ED52ED52FC0EDB2AFD0E01E3DB2AD9CF2F
:10585000E9FFDACFEAFFEECF0DF0EECF0EF0EECF9C
:105860000FF0EFCF10F0E80E126E030E136E146AF5
:10587000156ACCEC25F0040E0DC0DBFF050E0EC042
:10588000DBFF040EDBCF04F0050EDBCF05F0E80EE6
:105890000502F3CF05F0030E0402F3500526E80ECF
:1058A0000402F3CF04F0F4500526066A076AD9CF44
:1058B000E9FFDACFEAFF0450EE5C006E0550EE58C7
:1058C000016E0650EE58026E0750EE58036E00C08F
:1058D000DFFF010E01C0DBFF020E02C0DBFF030E83
:1058E00003C0DBFF300EE76E040EDBCF00F0050EC9
:1058F000DBCF01F0E7500026000E0122FC0EDBCFCB
:10590000E9FFFD0EDBCFEAFF00C0EFFFFC0EDB2A54
:10591000FD0E01E3DB2AFC0EDBCFE9FFFD0EDBCF42
:10592000EAFF2E0EEF6EFC0EDB2AFD0E01E3DB2AF2
:10593000640EF36E070EF3CFDBFF080EDB6A010E79
:10594000F36E060EF3CFDBFFD950070FE96EDACF07
:10595000EAFFEE50ED1001E193D0070EDBCF00F02F
:10596000080EDBCF01F0026A036A00C012F001C02A
:1059700013F002C014F003C015F0DFCF0DF0010EDC
:10598000DBCF0EF0020EDBCF0FF0030EDBCF10F0FB
:10599000CCEC25F0040E0DC0DBFF050E0EC0DBFFC6
:1059A000D950040FE96EDACFEAFFEE50ED100DE1A9
:1059B000060EDB500AE1D950070FE96EDACFEAFF95
:1059C000010EEE1801E1ED5019E1300EE76E040E04
:1059D000DBCF00F0050EDBCF01F0E7500026000E14
:1059E0000122FC0EDBCFE9FFFD0EDBCFEAFF00C09A
:1059F000EFFFFC0EDB2AFD0E01E3DB2A040EDBCFFA
:105A00000FF0050EDBCF10F0070EDBCF14F0080E01
:105A1000DBCF15F02DEC26F00DC004F00EC005F024
:105A2000066A076AD9CFE9FFDACFEAFF0450EE5CD5
:105A3000006E0550EE58016E0650EE58026E07508B
:105A4000EE58036E00C0DFFF010E01C0DBFF020E47
:105A500002C0DBFF030E03C0DBFFD950070FE96E66
:105A6000DACFEAFF0A0E146E156AEECF0FF0EDCF13
:105A700010F0B1EC21F00FC0EEFF10C0EDFF64D7C5
:105A8000FC0EDBCFE9FFFD0EDBCFEAFFEF6AD9CFDB
:0A5A9000E1FFE552E7CFD9FF120055
:065A9A00D9CFE6FFE1CFC9
:105AA000D9FF020EE126FE0EDB50EA6A000FE96E16
:105AB000050EEA22440EEF6EFE0EDB2A010EDB6AB3
:105AC000040EF36E010EDBCFF4FFF350F45C2EE214
:105AD000010EF36EDB5004E0D890F336E806FCE1EB
:105AE000F350010168151FE0010EDBCFE6FF2DEC3E
:105AF00024F0E552DF6EFE0EDB50EA6A000FE96E1D
:105B0000050EEA222C0EEF6EFE0EDB2A300EDF268B
:105B1000FE0EDB50EA6A000FE96E050EEA22DFCFC7
:105B2000EFFFFE0EDB2A010EDB2ACAD7FE0EDB508A
:105B3000EA6A000FE96E050EEA222C0EEF6EFE0EE9
:105B4000DB2ADB5000D0D9CFE1FFE552E7CFD9FF08
:105B50001200D9CFE6FFE1CFD9FF110EE1260C0EDE
:105B6000DB6AFE0EDB50EA6A000FE96E050EEA22E0
:105B7000410EEF6EFE0EDB2ADB50EA6A000FE96E83
:105B8000050EEA222C0EEF6EFE0EDB2A0F0EDB6AEC
:105B9000040EF36E0F0EDBCFF4FFF350F45C50E213
:105BA000010EF36E0F0EDB5004E0D890F336E806DA
:105BB000FCE1F3500101671540E0D950080FE66E93
:105BC000DACFE6FF0F0EDB28E66E6FEC2BF0E10676
:105BD000E106E106100EDB6A060EF36E100EDBCF57
:105BE000F4FFF350F45C1EE2D950080F006EDACFD8
:105BF00001F0100EDB500F01EA6B0024E96F015039
:105C0000EA23EF50E66EFE0EDB50EA6A000FE96E03
:105C1000050EEA22E552E750EF6E100EDB2AFE0E6B
:105C2000DB2ADAD7FE0EDB50EA6A000FE96E050EBA
:105C3000EA222C0EEF6EFE0EDB2A0F0EDB2AA8D70F
:105C4000FE0EDB5000D0D9CFE1FFE552E7CFD9FF00
:105C50001200D9CFE6FFE1CFD9FF030EE126D9CF5D
:105C6000E6FFDACFE6FF69EC25F0E552E5520009E0
:105C700001E1DFD001016A51DF5C01E0B7D00E0124
:105C8000235101E0AED09BEC21F001016B050E0128
:105C9000236F00019451EA6A000FE96E020EEA22B6
:105CA0000D0EEF6E942B960EE66E000EE66EC2ECB5
:105CB0003BF0E552E552010EDB6ADB50EA6A960FD3
:105CC000E96E000EEA22EF5016E0010EDB50EA6AA0
:105CD000960FE96E000EEA22EF50E66E010EDB50E1
:105CE000EA6A000FE96E050EEA22E552E750EF6E10
:105CF000010EDB2AE2D7010EDB50EA6A000FE96EE3
:105D0000050EEA222C0EEF6E010EDB2A020EDB6A74
:105D1000020EDB50EA6A000FE96E020EEA22EF5033
:105D20000D0818E0020EDB50EA6A000FE96E020E61
:105D3000EA22EF50E66E010EDB50EA6A000FE96ED0
:105D4000050EEA22E552E750EF6E020EDB2A010E45
:105D5000DB2ADED7010EDB50EA6A000FE96E050E82
:105D6000EA222C0EEF6E010EDB2ADBCFE6FF95DE7A
:105D7000E552E76E010EE7CFDBFFDBCFE6FFE9DEA2
:105D8000E552E76E010EE7CFDBFFDB06DB50EA6A88
:105D9000000FE96E050EEA220D0EEF6E010EDB2AF2
:105DA000DB50EA6A000FE96E050EEA220A0EEF6E7A
:105DB000010EDB2ADBCFE6FFE66A000EE66E050E7B
:105DC000E66E000EE66EE66ABEEC4CF0F56E060E70
:105DD000E15EF5500001946B946B956B9DEC21F0A6
:105DE00004D023070001946B956B23D00101695106
:105DF000DF5C05E10001010E956F946B1AD0000184
:105E0000955117E09451006E016A0150000AE8AE06
:105E100002D0D89004D07E0E005C000E015809E23A
:105E20009451EA6A000FE96E020EEA22DFCFEFFF1B
:105E3000942BD9CFE1FFE552E7CFD9FF1200D9CF9C
:105E4000E6FFE1CFD9FF020EE1269BEC21F0DF6AED
:105E5000DFCFE6FF22DEE552DF6EDFCFE6FF79DE41
:105E6000E552DF6E0001A6512AE0960EE66E000EA6
:105E7000E66EC2EC3BF0E552E552010EDB6ADB5008
:105E8000EA6A960FE96E000EEA22EF5016E0010E64
:105E9000DB50EA6A960FE96E000EEA22EF50E66EDA
:105EA000DF50EA6A000FE96E050EEA22E552E7507C
:105EB000EF6E010EDB2ADF2AE2D70001A66BDF506E
:105EC000EA6A000FE96E050EEA222C0EEF6EDF2A59
:105ED0000E01245127E0010EDB6ADB50EA6A000F55
:105EE000E96E020EEA22EF500D0816E0010EDB50BB
:105EF000EA6A000FE96E020EEA22EF50E66EDF500A
:105F0000EA6A000FE96E050EEA22E552E750EF6EED
:105F1000010EDB2ADF2AE1D7DF060001946B956BC7
:105F20000E01246BDF50EA6A000FE96E050EEA22CB
:105F30000D0EEF6EDF2ADF50EA6A000FE96E050EE4
:105F4000EA220A0EEF6EDF2A2951D880DF5402E2DE
:105F5000DFCF29FE2A5135E02E5133E0010EDB6AF6
:105F6000DF50F36E010EDBCFF4FFF350F45C18E268
:105F7000010EDB50EA6A000FE96E050EEA22EF50CF
:105F8000E66E000E2525E96E080E2621EA6EE55222
:105F9000E750EF6E252B000E2623010EDB2AE0D7FB
:105FA0002951016A2525006E26510122000ED88054
:105FB0000054010E015404E2010E2C6F2A6B2B6F6A
:105FC00036D02B5134E02F5132E0010EDB6ADF5026
:105FD000F36E010EDBCFF4FFF350F45C18E2010E18
:105FE000DB50EA6A000FE96E050EEA22EF50E66E1A
:105FF000000E2725E96E090E2821EA6EE552E750CA
:10600000EF6E272B000E2823010EDB2AE0D7295143
:10601000016A2725006E28510122000ED880005405
:10602000010E015404E2010E2D6F2B6B2A6F9DECC3
:1060300021F0D9CFE1FFE552E7CFD9FF1200D9CF48
:10604000E6FFE1CFD9FFE652D9CFE6FFDACFE6FF90
:1060500069EC25F0E552E552000941E001016A5181
:10606000DF5C1AE10E01235112E101016B050E0103
:10607000236F00019451EA6A000FE96E020EEA22D2
:106080000D0EEF6E942B0E01010E246F04D023072A
:106090000001946B956B23D001016951DF5C05E130
:1060A0000001010E956F946B1AD00001955117E015
:1060B0009451006E016A0150000AE8AE02D0D890F7
:1060C00004D07E0E005C000E015809E29451EA6A89
:1060D000000FE96E020EEA22DFCFEFFF942BE552AC
:1060E000E552E7CFD9FF120008EC22F0F28EF29CC5
:1060F000E66AE66AAEEC23F0E552E552E66A010E86
:10610000E66EAEEC23F0E552E552E66A020EE66E6C
:10611000AEEC23F0E552E552E66A030EE66EAEEC15
:1061200023F0E552E552010EE66EE66AE0EC23F05C
:10613000E552E552010EE66EE66EE0EC23F0E55224
:10614000E552010EE66E020EE66EE0EC23F0E5523B
:10615000E552010EE66E030EE66EE0EC23F0E5522A
:10616000E552E66A170EE66E59EC24F0E552E55268
:106170003CEC33F030EC23F05CEC41F0E66AE66A8C
:10618000E0EC23F0E552E552E66A010EE66EE0EC43
:1061900023F0E552E552E66A020EE66EE0EC23F0EB
:1061A000E552E552E66A030EE66EE0EC23F0E552B6
:1061B000E552010EE66EE66AAEEC23F0E552E552DA
:1061C000010EE66EE66EAEEC23F0E552E552010EEE
:1061D000E66E020EE66EAEEC23F0E552E552010EDD
:1061E000E66E030EE66EAEEC23F0E552E552F19E4C
:1061F0000001946B956B0D0EE66E0E0EE66ECCEC08
:1062000027F0E552E55281EC38F0DDEC38F0CDECCA
:1062100039F0960EE66E000EE66EC2EC3BF0E552EB
:10622000E552C60ED56EF184D76AB90ED66EF294D9
:10623000F28A00019C6B9D6B9E6B9F6BA06BA56BA4
:106240000E01010E306F3CEC23F060EC41F00009D0
:106250006BE00001010EA56F01016C5105E000012A
:106260009C5102E0F6DC5FD09D0EE96E000EEA6EF6
:1062700001016D51EE5C6E51EE586F51EE58705148
:10628000EE584EE3C80E0001A15D000EA259000EAB
:10629000A359000EA45906E3010EA66FA16BA26BD1
:1062A000A36BA46B9C5101E0CADD0E012C5118E0D8
:1062B0002E6B2C6B25CEE6FF26CEE6FF000EE66E9B
:1062C000080EE66E000EE66EE66ABEEC4CF0F56E69
:1062D000060EE15EF5500E01010E2E6F256B266B4A
:1062E0002D5118E02F6B2D6B27CEE6FF28CEE6FF51
:1062F000000EE66E090EE66E000EE66EE66ABEEC75
:106300004CF0F56E060EE15EF5500E01010E2F6F9A
:10631000276B286B00019D6B9E6B9F6BA06B03D05E
:106320008EDE16EC2AF00CD00001A56B946B956BF9
:106330009C6B3AEC25F00E01010E306F14EC2AF044
:1063400000019C5127E1000EE66E0E0EE66E4FEC4A
:1063500051F0E552E55200019C6F9C511BE00E018B
:10636000305118E0306BBBEC51F039EC29F067C1CB
:10637000E6FF7F0EE66E010EE66EDEEC29F0E1062A
:10638000E106E10673C1E6FF71C1E6FF11EC25F0FD
:10639000E552E55201016C5105E000019C5102E01B
:1063A00016EC2AF050D7F29AD76AB90ED66E0001D1
:1063B000A5510CE000019D2B000E9E239F23A023DE
:1063C0000001A12B000EA223A323A423F294F28A9E
:1063D00011001200F2B4D3EF31F09EBAAEEF25F007
:1063E0009DA803D09EB891EF25F0A4BAF3EF24F056
:0A63F000A4B8D6EF24F0110012004B
:0663FA00D9CFE6FFE1CF60
:10640000D9FFE6528450100B04E18450080B01E1DF
:10641000F9D71F0E8416FE0EDB50E00B8412849019
:10642000000000008350DF6E8480DF5000D0E55212
:10643000E552E7CFD9FF1200D9CFE6FFE1CFD9FF70
:106440008450100B04E18450080B01E1F9D7FD0ED4
:10645000DB50836E1F0E8416FE0EDB50E00B8412A1
:106460008492000000008482E552E7CFD9FF120039
:10647000D9CFE6FFE1CFD9FFFE0EDB380F0BF36E6D
:10648000FE0EF3CFDBFFDB5009080BE2370E006E88
:10649000FE0EDBCFE7FF0050E726FE0EE7CFDBFF67
:1064A0000AD0300E006EFE0EDBCFE7FF0050E7266D
:1064B000FE0EE7CFDBFFFE0EDBCFE6FF8DEC24F018
:1064C000E552000901E1F7D7E552E7CFD9FF120005
:1064D000D9CFE6FFE1CFD9FFFE0EDB98DB9ADB9C3C
:1064E000DB9EFE0EDB5009080BE2370E006EFE0E3F
:1064F000DBCFE7FF0050E726FE0EE7CFDBFF0AD039
:10650000300E006EFE0EDBCFE7FF0050E726FE0EDA
:10651000E7CFDBFFFE0EDBCFE6FF8DEC24F0E5528C
:10652000000901E1F7D7E552E7CFD9FF1200D9CF33
:10653000E6FFE1CFD9FF030EE126FD0EDBCF0FF022
:10654000FE0EDBCF10F0DE520FC0DEFF10C0DDFF0D
:10655000DD52DF6A100EDF5C3AE2FD0EDBCFE9FFB1
:10656000FE0EDBCFEAFFEF50E66E82DFE552FD0E56
:10657000DBCFE9FFFE0EDBCFEAFFEF50E66EA8DFD0
:10658000E552FD0EDB2AFE0E01E3DB2AFD0EDBCF1A
:10659000E9FFFE0EDBCFEAFFEF50E66E69DFE55262
:1065A000FD0EDBCFE9FFFE0EDBCFEAFFEF50E66E1C
:1065B0008FDFE552FD0EDB2AFE0E01E3DB2A200E03
:1065C000E66E91EC27F0E552020EDF26C3D7010EEE
:1065D000DBCF0FF0020EDBCF10F0FD0E0FC0DBFFA4
:1065E000FE0E10C0DBFFDF6A100EDF5C2CE2FD0E3A
:1065F000DBCFE9FFFE0EDBCFEAFFEFCF00F0200E8E
:10660000005C15E3FD0EDBCFE9FFFE0EDBCFEAFFFA
:10661000EF507E080CE3FD0EDBCFE9FFFE0EDBCF73
:10662000EAFFEF50E66E91EC27F0E55205D02E0E12
:10663000E66E91EC27F0E552FD0EDB2AFE0E01E33B
:10664000DB2ADF2AD1D70D0EE66E91EC27F0E5525A
:106650000A0EE66E91EC27F0E552D9CFE1FFE55244
:10666000E7CFD9FF120084A603D08588000E03D09F
:106670008598FF0E00D01200858897988494969490
:10668000848096908482969296869688836A956A8C
:106690001F0E8416961685981200D9CFE6FFE1CF1B
:1066A000D9FF140EE126130EDB6ADDDF000901E1DC
:1066B00098D0956AE00EE66EC00EE66EBDDEE5523D
:1066C000E552E66AA00EE66EB7DEE552E552FD0E33
:1066D000DBCF00F0FE0EDBCF01F001C000F0016A5D
:1066E0000050E66E800EE66EA7DEE552E552FF0E24
:1066F000E76EFD0EDBCF00F0FE0EDBCF01F0E750C2
:106700000016016A0050E66E600EE66E95DEE552F8
:10671000E552010EE66E400EE66E8EDEE552E55263
:10672000200EE66EE00EE66E87DEE552E5529568D5
:106730001F0E8416100EDB6A110EDB6A120EDB6A66
:10674000110EDBCF00F0120EDBCF01F0000E005C6B
:10675000020E015844E2E66A50DEE552E66ED9CFF9
:1067600000F0DACF01F0100EDB500F01EA6B0024CD
:10677000E96F0150EA23E552E750EF6E100EDB2A75
:10678000110EDB2A120E01E3DB2AE66A36DEE55241
:10679000E66ED9CF00F0DACF01F0100EDB500F011A
:1067A000EA6B0024E96F0150EA23E552E750EF6EEF
:1067B000100EDB2AF36EDBCFF4FFF350F45C09E339
:1067C000D9CFE6FFDACFE6FFB2DEE552E552100E92
:1067D000DB6A110EDB2A120E01E3DB2AB1D7956AC0
:1067E00005D0010EF36E130EF3CFDBFF130EDB505B
:1067F00000D0D9CFE1FFE552E7CFD9FF1200D9CFC2
:10680000E6FFE1CFD9FF160EE126150EDB6A2BDF7E
:10681000000966E0956AEC0EE66EE00EE66E0CDEB0
:10682000E552E55295681F0E8416040EDB6ADE6A97
:10683000DD6ADECF00F0DDCF01F0000E005C020E5D
:1068400001584CE2E66AD9DDE552E76E030EE7CF68
:10685000DBFFDF2A010E01E3DB2AE66ACEDDE5522B
:10686000E76E020EE7CFDBFFD950050F006EDACFDF
:1068700001F0040EDB500F01EA6B0024E96F0150B8
:10688000EA23020EDBCFEFFF040EDB2AD950050FFF
:10689000006EDACF01F0040EDB50EA6B0024E96FE2
:1068A0000150EA23030EDBCFEFFF040EDB2A100EAC
:1068B000F36E040EDBCFF4FFF350F45C0AE3D9501F
:1068C000050FE66EDACFE6FF32DEE552E552040E42
:1068D000DB6ADF2A010E01E3DB2AABD7956A05D01C
:1068E000010EF36E150EF3CFDBFF150EDB5000D05B
:1068F000D9CFE1FFE552E7CFD9FF1200D9CFE6FFAC
:10690000E1CFD9FF040EE126030EDB6AACDE0009FD
:106910005CE0956AE00EE66EC00EE66E8DDDE55237
:10692000E552E66AA00EE66E87DDE552E552FD0E01
:10693000DBCF00F0FE0EDBCF01F001C000F0016AFA
:106940000050E66E800EE66E77DDE552E552FF0EF2
:10695000E76EFD0EDBCF00F0FE0EDBCF01F0E7505F
:106960000016016A0050E66E600EE66E65DDE552C7
:10697000E552010EE66E400EE66E5EDDE552E55232
:10698000300EE66EE00EE66E57DDE552E5521F0E64
:106990008416020EDB6ADE6ADD6ADECF00F0DDCF30
:1069A00001F0000E005C020E01580EE2020EDBCF79
:1069B000E6FFE66A41DDE552E552020EDB2ADF2AF8
:1069C000010E01E3DB2AE9D705D0010EF36E030EB9
:1069D000F3CFDBFF030EDB5000D0D9CFE1FFE55250
:1069E000E7CFD9FF1200D9CFE6FFE1CFD9FF060EDE
:1069F000E126010EF36E030EF3CFDBFF020EDB6A1E
:106A0000660E006E660E016E0050011001E1EDD0C1
:106A1000030EDB5001E1B5D08450080B01E0B1D08A
:106A2000956AE00EE66EC00EE66E06DDE552E552B2
:106A3000E66AA00EE66E00DDE552E552FD0EDBCF04
:106A400000F0FE0EDBCF01F001C000F0016A005043
:106A5000E66E800EE66EF0DCE552E552FF0EE76E64
:106A6000FD0EDBCF00F0FE0EDBCF01F0E75000168D
:106A7000016A0050E66E600EE66EDEDCE552E5521D
:106A8000010EE66E400EE66ED7DCE552E5529568E3
:106A9000C00EE66EB2DCE552200FE66ED950040F50
:106AA000E96EDACFEAFFE552E750EE6EED6AA00E2E
:106AB000E66EA3DCE552006E016AD950040FE96E60
:106AC000DACFEAFF0050EE260150ED22FD0EDBCFBB
:106AD00002F0FE0EDBCF03F003C002F0036A02C037
:106AE000E6FF800EE66E89DCE552E552E7CF02F064
:106AF000D8800254006E016AD950040FE96EDACFD3
:106B0000EAFF0050EE260150ED22FF0EE76EFD0E6B
:106B1000DBCF02F0FE0EDBCF03F0E7500216036A74
:106B200002C0E6FF600EE66E68DCE552E552E7CF94
:106B300002F0D8800254006E016AD950040FE96E49
:106B4000DACFEAFF0050EE260150ED22400EE66E4D
:106B500054DCE552FF0F006E016AD950040FE96E54
:106B6000DACFEAFF0050EE260150ED22D950040F93
:106B7000E96EDACFEAFFEE50ED1002E1030EDB6AB8
:106B800047D7956A200EE66EE00EE66E55DCE552BC
:106B9000E55295681F0E8416DE6ADD6ADECF00F0CE
:106BA000DDCF01F0FB0EDBCF02F0FC0EDBCF03F0FC
:106BB0000250005C0350015817E2E66A1EDCE55201
:106BC000E66EF90EDBCFE9FFFA0EDBCFEAFFE55206
:106BD000E750EF6EF90EDB2AFA0E01E3DB2ADF2A1B
:106BE000010E01E3DB2ADAD705D0010EF36E020EA7
:106BF000F3CFDBFF020EDB5000D0D9CFE1FFE5522F
:106C0000E7CFD9FF1200D9CFE6FFE1CFD9FF030EBE
:106C1000E126020EDB6A660E006E660E016E005003
:106C200001102AE0DE6ADD6ADECF00F0DDCF01F080
:106C3000FD0EDBCF02F0FE0EDBCF03F00250005C56
:106C40000350015818E2E66AFDEC31F0E552E66EB9
:106C5000FB0EDBCFE9FFFC0EDBCFEAFFE552E7508E
:106C6000EF6EFB0EDB2AFC0E01E3DB2ADF2A010EAE
:106C700001E3DB2AD9D705D0010EF36E020EF3CF64
:106C8000DBFF020EDB5000D0D9CFE1FFE552E7CFAA
:106C9000D9FF1200D9CFE6FFE1CFD9FFE652DF6A74
:106CA000660E006E660E016E0050011007E0200EA9
:106CB000E66EFDEC31F0E552DF6E02D0010EDF6EC4
:106CC000DF5000D0E552E552E7CFD9FF1200D9CF0F
:106CD000E6FFE1CFD9FF020EE126010EDB6A660E68
:106CE000006E660E016E0050011010E0E00EE66EC0
:106CF000FDEC31F0E552DF6EDF1C800B06E0010E8B
:106D0000DF1403E0DE52020EDD6E03D0DE52010E10
:106D1000DD6E010EDB5000D0D9CFE1FFE552E7CFA9
:106D2000D9FF1200D9CFE6FFE1CFD9FF060EE12649
:106D3000010EF36E030EF3CFDBFF020EDB6A660E6D
:106D4000006E660E016E0050011001E1F7D0030ED7
:106D5000DB5001E1BFD08450080B01E0BBD0956A45
:106D6000E00EE66EC00EE66E1CEC32F0E552E55227
:106D7000E66AA00EE66E1CEC32F0E552E552FD0E1E
:106D8000DBCF00F0FE0EDBCF01F001C000F0016AA6
:106D90000050E66E800EE66E1CEC32F0E552E552D5
:106DA000FF0EE76EFD0EDBCF00F0FE0EDBCF01F035
:106DB000E7500016016A0050E66E600EE66E1CECAD
:106DC00032F0E552E552010EE66E400EE66E1CEC26
:106DD00032F0E552E5529568C00EE66EFDEC31F0FA
:106DE000E552200FE66ED950040FE96EDACFEAFFC4
:106DF000E552E750EE6EED6AA00EE66EFDEC31F066
:106E0000E552006E016AD950040FE96EDACFEAFF4D
:106E10000050EE260150ED22FD0EDBCF02F0FE0EFB
:106E2000DBCF03F003C002F0036A02C0E6FF800E6E
:106E3000E66EFDEC31F0E552E552E7CF02F0D88086
:106E40000254006E016AD950040FE96EDACFEAFFEE
:106E50000050EE260150ED22FF0EE76EFD0EDBCF57
:106E600002F0FE0EDBCF03F0E7500216036A02C009
:106E7000E6FF600EE66EFDEC31F0E552E552E7CF3D
:106E800002F0D8800254006E016AD950040FE96EF6
:106E9000DACFEAFF0050EE260150ED22400EE66EFA
:106EA000FDEC31F0E552FF0F006E016AD950040F7E
:106EB000E96EDACFEAFF0050EE260150ED22D950FC
:106EC000040FE96EDACFEAFFEE50ED1002E1030E97
:106ED000DB6A3DD7956A300EE66EE00EE66E1CEC7E
:106EE00032F0E552E5521F0E8416DE6ADD6ADECF0F
:106EF00000F0DDCF01F0FB0EDBCF02F0FC0EDBCFAC
:106F000003F00250005C0350015817E2F90EDBCF8A
:106F1000E9FFFA0EDBCFEAFFEF50E66EE66A1CEC03
:106F200032F0E552E552F90EDB2AFA0E01E3DB2AD4
:106F3000DF2A010E01E3DB2ADAD705D0010EF36E5A
:106F4000020EF3CFDBFF020EDB5000D0D9CFE1FF02
:106F5000E552E7CFD9FF1200D9CFE6FFE1CFD9FF45
:106F6000030EE126020EDB6A660E006E660E016EEF
:106F70000050011029E0DE6ADD6ADECF00F0DDCFCF
:106F800001F0FD0EDBCF02F0FE0EDBCF03F002506E
:106F9000005C0350015817E2FB0EDBCFE9FFFC0E4B
:106FA000DBCFEAFFEF50E66EE66A1CEC32F0E5520A
:106FB000E552FB0EDB2AFC0E01E3DB2ADF2A010E81
:106FC00001E3DB2ADAD705D0010EF36E020EF3CF10
:106FD000DBFF020EDB5000D0D9CFE1FFE552E7CF57
:046FE000D9FF1200C3
:0C6FE4000000000000000000120082927B
:106FF000F9DF829012008292F5DF8280F3DF8282D5
:107000001200D9CFE6FFE1CFD9FF020EE126010E33
:10701000DF6EDB6A080EF36E010EDBCFF4FFF35078
:10702000F45C20E2010EDBCFE6FF070EE552D880CC
:10703000E754006EFE0EDB5000C0E7FFE75204E0AD
:10704000E8427F0BE706FCE1010BF36EF346FD0E11
:107050008214F310826EC6DF8280C4DF8290010E3C
:10706000DB2AD8D79482BEDF8280BCDF8250020B3D
:1070700001E0010EDF6E82909492DF5002E1FF0E7C
:1070800002D0000E00D0D9CFE1FFE552E7CFD9FF03
:107090001200D9CFE6FFE1CFD9FF020EE12694829C
:1070A0008290A0DF010EDB6A080EF36E010EDBCFCB
:1070B000F4FFF350F45C0EE2DF9EDF46828092DF45
:1070C0008250020B01E0010EDF2682908BDF010E61
:1070D000DB2AEAD79492FE0EDB50010B010BF36E14
:1070E000F346FD0E8214F310826E7CDF82807ADF1D
:1070F0008290DF5000D0D9CFE1FFE552E7CFD9FF32
:107100001200D9CFE6FFE1CFD9FF160EE126D00E4F
:10711000DF6E020EDB6A030EDB6AD950040FE96EE4
:10712000DACFEAFF0A0EEE6E0D0EEE6E490EEE6E2F
:107130006E0EEE6E690EEE6E740EEE6E690EEE6EF3
:10714000610EEE6E6C0EEE6E690EEE6E730EEE6EEE
:10715000650EEE6E640EEE6E200EEE6E520EEE6E4C
:10716000540EEE6E430EEE6EEE6A94909492829000
:107170008282828037DF3BDFDFCFE6FF42DFE552EE
:10718000E76E020EE7CFDBFFDB5009E0030EDBCF3B
:10719000E6FF37DFE552E76E020EE7CFDBFF2BDFBE
:1071A000020EDB5002E0FF0E02D0000E00D0D9CF5D
:1071B000E1FFE552E7CFD9FF1200D9CFE6FFE1CFDB
:1071C000D9FF030EE126D10EDF6E010EDB6AF36EEE
:1071D000020EF3CFDBFF95DF0ADFDFCFE6FF11DF23
:1071E000E552E76E020EE7CFDBFFDB5033E0010E26
:1071F000DBCFE6FF4EDFE5520001BD6F010EDBCFB6
:10720000E6FF47DFE5520001BE6F010EDBCFE6FF70
:1072100040DFE5520001BF6F010EDBCFE6FF39DF33
:10722000E5520001C06F010EDBCFE6FF32DFE55211
:107230000001C16F010EDBCFE6FF2BDFE55200013D
:10724000C26FDE52010EDD6EDBCFE6FF22DFE552BC
:107250000001C36FD0DED9CFE1FFE552E7CFD9FF00
:107260001200D9CFE6FFE1CFD9FF0B0EE126D00EF9
:10727000DF6EDE52010EDD6E030EDB6A020EDB6A8C
:10728000FD0EDBCFE9FFFE0EDBCFEAFFEF504CE057
:10729000FD0EDBCFE9FFFE0EDBCFEAFFEF50D00F94
:1072A000E66ED950040F006EDACF01F0020EDB500B
:1072B0000F01EA6B0024E96F0150EA23E552E75021
:1072C000EF6ED950040F006EDACF01F0020EDB50E2
:1072D000EA6B0024E96F0150EA23EF38F00BEF6E00
:1072E000FD0EDB2AFE0E01E3DB2AFD0EDBCFE9FFFC
:1072F000FE0EDBCFEAFFEF50D00F026ED950040F25
:10730000006EDACF01F0020EDB50EA6B0024E96F69
:107310000150EA230250EF26FD0EDB2AFE0E01E3A8
:10732000DB2A020EDB2AACD762DEDFCFE6FF69DEA6
:10733000E552E76E010EE7CFDBFFDB5009E0030EFD
:10734000DBCFE6FF5EDEE552E76E010EE7CFDBFF47
:10735000020EDB6A070EF36E020EDBCFF4FFF35072
:10736000F45C14E2D950040F006EDACF01F0020E83
:10737000DB500F01EA6B0024E96F0150EA23EF5064
:10738000E66E3FDEE552020EDB2AE4D734DED9CFCB
:10739000E1FFE552E7CFD9FF1200D9CFE6FFE1CFF9
:1073A000D9FF2D0EE126D9CFE9FFDACFEAFF0A0E89
:1073B000EE6E0D0EEE6E430EEE6E6F0EEE6E6E0EF8
:1073C000EE6E730EEE6E740EEE6E720EEE6E750E47
:1073D000EE6E630EEE6E740EEE6E690EEE6E6E0E57
:1073E000EE6E670EEE6E200EEE6E440EEE6E610EC9
:1073F000EE6E740EEE6E650EEE6E200EEE6E610E8B
:10740000EE6E6E0EEE6E640EEE6E200EEE6E540E8E
:10741000EE6E690EEE6E6D0EEE6E650EEE6E0A0E7F
:10742000EE6E0D0EEE6EEE6A0001BD390F0B0A0D09
:10743000F350E66ED9501F0FE96EDACFEAFFE5523E
:10744000E750EE6EED6A0F0EBD15006E016AD95061
:107450001F0FE96EDACFEAFF0050EE260150ED2251
:10746000BE390F0B0A0DF350E66ED950210FE96EAD
:10747000DACFEAFFE552E750EE6EED6A0F0EBE1569
:10748000006E016AD950210FE96EDACFEAFF005091
:10749000EE260150ED22BF390F0B030B0A0DF350FE
:1074A000E66ED950230FE96EDACFEAFFE552E750D6
:1074B000EE6EED6A0F0EBF15006E016AD950230FF4
:1074C000E96EDACFEAFF0050EE260150ED22C13915
:1074D0000F0B0A0DF350E66ED950270FE96EDACF85
:1074E000EAFFE552E750EE6EED6A0F0EC115006E31
:1074F000016AD950270FE96EDACFEAFF0050EE2675
:107500000150ED22C2390F0B010B0A0DF350E66E4C
:10751000D950290FE96EDACFEAFFE552E750EE6E57
:10752000ED6A0F0EC215006E016AD950290FE96E7F
:10753000DACFEAFF0050EE260150ED22C3390F0BDF
:107540000A0DF350E66ED9502B0FE96EDACFEAFF41
:10755000E552E750EE6EED6A0F0EC315006E016A3C
:10756000D9502B0FE96EDACFEAFF0050EE2601501A
:10757000ED22D9502B0FE96EDACFEAFFD00EEE26BE
:10758000070EED22D9501F0FE96EDACFEAFF090E80
:10759000D880EE54000EED5413E3300EC46FC50EC8
:1075A000E66E000EE66E1F0EDBCFE6FF200EDBCF91
:1075B000E6FF94EC26F0E106E106E106E10610D0D4
:1075C000C40EE66E000EE66E1F0EDBCFE6FF200E49
:1075D000DBCFE6FF94EC26F0E106E106E106E106EA
:1075E000D950210FE96EDACFEAFF090ED880EE54A8
:1075F000000EED5414E30001300EC66FC70EE66EA8
:10760000000EE66E210EDBCFE6FF220EDBCFE6FF9B
:1076100094EC26F0E106E106E106E10610D0C60E84
:10762000E66E000EE66E210EDBCFE6FF220EDBCF0C
:10763000E6FF94EC26F0E106E106E106E106D9500A
:10764000230FE96EDACFEAFF090ED880EE54000E60
:10765000ED5414E30001300EC86FC90EE66E000E43
:10766000E66E230EDBCFE6FF240EDBCFE6FF94ECC5
:1076700026F0E106E106E106E10610D0C80EE66E4E
:10768000000EE66E230EDBCFE6FF240EDBCFE6FF17
:1076900094EC26F0E106E106E106E106D950270F59
:1076A000E96EDACFEAFF090ED880EE54000EED54F1
:1076B00014E30001300ECA6FCB0EE66E000EE66ECC
:1076C000270EDBCFE6FF280EDBCFE6FF94EC26F09B
:1076D000E106E106E106E10610D0CA0EE66E000EF4
:1076E000E66E270EDBCFE6FF280EDBCFE6FF94EC3D
:1076F00026F0E106E106E106E106D950290FE96E20
:10770000DACFEAFF090ED880EE54000EED5414E3F0
:107710000001300ECC6FCD0EE66E000EE66E290E27
:10772000DBCFE6FF2A0EDBCFE6FF94EC26F0E10686
:10773000E106E106E10610D0CC0EE66E000EE66E24
:10774000290EDBCFE6FF2A0EDBCFE6FF94EC26F016
:10775000E106E106E106E106CE0EE66E000EE66EFB
:107760002B0EDBCFE6FF2C0EDBCFE6FF94EC26F0F2
:10777000E106E106E106E106D9CFE1FFE552E7CFF8
:10778000D9FF1200D9CFE6FFE1CFD9FF060EE126DF
:10779000B8DC13DD0001BF390F0B030B0A0DF3CF6B
:1077A00000F0016A026A00C0DFFF010E01C0DBFFCA
:1077B000020E02C0DBFFD9CFE9FFDACFEAFF100EDD
:1077C000136E0E0E146E156AEECF0EF0EECF0FF0A4
:1077D000EFCF10F04BEC26F00DC0EDFF0CC0EDFF2D
:1077E0000BC0EFFF0F0E0001BF15006E016A026AA9
:1077F000030E00C0DBFF040E01C0DBFF050E02C05C
:10780000DBFFD950030FE96EDACFEAFF100E136EDB
:107810000E0E146E156AEECF0EF0EECF0FF0EFCF16
:1078200010F04BEC26F00DC0EDFF0CC0EDFF0BC0CF
:10783000EFFFD9CFE9FFDACFEAFF030EDB50EE26E8
:10784000040EDB50EE22050EDB50EE220001BE39A5
:107850000F0B0A0DF3CF00F0016A026A030E00C09D
:10786000DBFF040E01C0DBFF050E02C0DBFF0F0EC5
:10787000BE15006E016A026AD950030FE96EDACFB5
:10788000EAFF0050EE260150EE220250EE22D950BF
:10789000030FE96EDACFEAFF3C0E136E146A156A25
:1078A000EECF0EF0EECF0FF0EFCF10F04BEC26F056
:1078B0000DC0EDFF0CC0EDFF0BC0EFFFD9CFE9FF0E
:1078C000DACFEAFF030EDB50EE26040EDB50EE2289
:1078D000050EDB50EE220001BD390F0B0A0DF3CF70
:1078E00000F0016A026AD9CFE9FFDACFEAFF00505F
:1078F000EE260150EE220250EE220F0EBD15006E54
:10790000016A026AD9CFE9FFDACFEAFF0050EE261A
:107910000150EE220250EE22FD0EDBCFE6FFFE0EFE
:10792000DBCFE6FFD9CFE9FFDACFEAFFEECFE6FF04
:10793000EECFE6FFEFCFE6FF62EC28F0F56E050E26
:10794000E15EF550D9CFE1FFE552E7CFD9FF120054
:10795000D9CFE6FFE1CFD9FF2D0EE126D9CFE9FF40
:10796000DACFEAFF0A0EEE6E0D0EEE6E430EEE6EED
:107970006F0EEE6E6E0EEE6E730EEE6E740EEE6E9B
:10798000720EEE6E750EEE6E630EEE6E740EEE6E91
:10799000690EEE6E6E0EEE6E670EEE6E200EEE6EE1
:1079A000440EEE6E610EEE6E740EEE6E650EEE6EB1
:1079B000200EEE6E610EEE6E6E0EEE6E640EEE6ECC
:1079C000200EEE6E540EEE6E690EEE6E6D0EEE6EC5
:1079D000650EEE6E0A0EEE6E0D0EEE6EEE6A81EC28
:1079E00038F0DDEC38F00001BD390F0B0A0DF35013
:1079F000E66ED9501F0FE96EDACFEAFFE552E75085
:107A0000EE6EED6A0F0EBD15006E016AD9501F0FA4
:107A1000E96EDACFEAFF0050EE260150ED22BE39C2
:107A20000F0B0A0DF350E66ED950210FE96EDACF35
:107A3000EAFFE552E750EE6EED6A0F0EBE15006EDE
:107A4000016AD950210FE96EDACFEAFF0050EE2625
:107A50000150ED22BF390F0B030B0A0DF350E66EF8
:107A6000D950230FE96EDACFEAFFE552E750EE6E08
:107A7000ED6A0F0EBF15006E016AD950230FE96E33
:107A8000DACFEAFF0050EE260150ED22C1390F0B8C
:107A90000A0DF350E66ED950270FE96EDACFEAFFF0
:107AA000E552E750EE6EED6A0F0EC115006E016AE9
:107AB000D950270FE96EDACFEAFF0050EE260150C9
:107AC000ED22C2390F0B010B0A0DF350E66ED950AF
:107AD000290FE96EDACFEAFFE552E750EE6EED6A64
:107AE0000F0EC215006E016AD950290FE96EDACF68
:107AF000EAFF0050EE260150ED22C3390F0B0A0DAC
:107B0000F350E66ED9502B0FE96EDACFEAFFE5525B
:107B1000E750EE6EED6A0F0EC315006E016AD95084
:107B20002B0FE96EDACFEAFF0050EE260150ED226E
:107B3000D9502B0FE96EDACFEAFFD00EEE26070EF2
:107B4000ED22D9CFE6FFDACFE6FFCCEC27F0E55205
:107B5000E552230EDBCFE6FF240EDBCFE6FFECEC95
:107B600027F0E552E5523A0EE66E91EC27F0E55229
:107B7000D950210FE96EDACFEAFF090ED880EE5412
:107B8000000EED5405E3300EE66E91EC27F0E55261
:107B9000210EDBCFE6FF220EDBCFE6FFECEC27F079
:107BA000E552E5523A0EE66E91EC27F0E552D950D7
:107BB0001F0FE96EDACFEAFF090ED880EE54000EEF
:107BC000ED5405E3300EE66E91EC27F0E5521F0E02
:107BD000DBCFE6FF200EDBCFE6FFECEC27F0E55233
:107BE000E552200EE66E91EC27F0E552270EDBCF32
:107BF000E6FF280EDBCFE6FFECEC27F0E552E5527E
:107C00002D0EE66E91EC27F0E552290EDBCFE6FF54
:107C10002A0EDBCFE6FFECEC27F0E552E5522D0E05
:107C2000E66E91EC27F0E5522B0EDBCFE6FF2C0E33
:107C3000DBCFE6FFECEC27F0E552E552D9CFE1FFD0
:087C4000E552E7CFD9FF120065
:087C4800D9CFE6FFE1CFD9FF1F
:107C5000E652DF6A100EDF5C1EE2DF50EA6A930F25
:107C6000E96E0E0EEA22EF50E66EA2EC27F0E55226
:107C7000DF2ADF50EA6A930FE96E0E0EEA22EF5018
:107C8000E66EA2EC27F0E552DF2A200EE66E91ECBC
:107C900027F0E552DFD70D0EE66E91EC27F0E552A6
:107CA0000A0EE66E91EC27F0E552E552E552E7CF79
:107CB000D9FF1200D9CFE6FFE1CFD9FFE6520E017E
:107CC000B56B930EE66E0E0EE66E100EE66EE66A6D
:107CD000000EE66EE66AF3EC34F0F56E060EE15E39
:107CE000F550010EDF6E1C0EDF5C0FE2930EE66EA8
:107CF0000E0EE66E100EE66EE66A03EC36F0E10656
:107D0000E106E106E106DF2AEED7800E0E01A15D55
:107D100020E1010EB56F930EE66E0E0EE66E100EAC
:107D2000E66EE66A03EC36F0E106E106E106E106FE
:107D3000040E0E01955D06E0060E955D03E00E0E45
:107D4000955D05E199CEA3FE9ACEA4FE01D0B56B58
:107D500004D0010EB56FA36BA46BB55166E0930E12
:107D6000E66E0E0EE66E100EE66EE66AA3CEE6FF37
:107D7000A4CEE6FFF3EC34F0F56E060EE15EF550AE
:107D80009ECEB0FE9FCEB1FEA0CEB2FEA1CEB3FE7F
:107D9000A2CEB4FE930EE66E0E0EE66E100EE66EEA
:107DA000E66A03EC36F0E106E106E106E10693CE71
:107DB000A5FE94CEA6FE95CEA7FE99CEAAFE9ACE9B
:107DC000ABFEAACE02F0ABCE03F0D890023603365B
:107DD00002500E01A325006E0350A421016E005035
:107DE000B325AC6F0150B421AD6FA6CE00F0A7CE85
:107DF00001F0050ED89000360136E806FBE100C020
:107E00000FF001C010F0B0CE14F0B1CE15F0B1EC0F
:107E100021F00FC0A8FE10C0A9FE0E01AC51A8258C
:107E2000AE6FAD51A921AF6F00D0E552E552E7CF5B
:107E3000D9FF1200D9CFE6FFE1CFD9FF0C0EE12622
:107E4000FD0EDBCF0FF0FE0EDBCF10F0020E0FC0E9
:107E5000DBFF030E10C0DBFF0E01A351B325006E44
:107E6000A451B421016E00C0DEFF01C0DDFFFD0E94
:107E7000DBCF00F0FE0EDBCF01F0000E005C010E48
:107E8000015814E3D950FD0FE96EFF0EDA20EA6EB7
:107E9000EE52ED06D950040FE96EDACFEAFFEE524A
:107EA000ED2ADF2A010E01E3DB2AE1D7930EE66E0D
:107EB0000E0EE66E100EE66EE66ADECFE6FFDDCF52
:107EC000E6FFF3EC34F0F56E060EE15EF550040EBD
:107ED000DB6A050EDB6AFD0EDBCF00F0FE0EDBCFAA
:107EE00001F0080E005C000E015821E3D950FD0F8F
:107EF000E96EFF0EDA20EA6E080EEE5E000EED5A15
:107F0000930EE66E0E0EE66E100EE66EE66A03EC5B
:107F100036F0E106E106E106E106D950040FE96E0C
:107F2000DACFEAFF080EEE26000EED22D4D7FD0EC2
:107F3000DBCFE9FFFE0EDBCFEAFFD890E936EA3669
:107F4000930EE9260E0EEA22020EEECFDBFF030EA1
:107F5000EDCFDBFFD950020FE96EDACFEAFFEECFAB
:107F600000F0EFCF01F0026A036A080E00C0DBFFE9
:107F7000090E01C0DBFF0A0E02C0DBFF0B0E03C0BF
:107F8000DBFFD950080FE96EDACFEAFFEF0ED88099
:107F9000EE54FF0EEE54000EEE54000EEE5405E2C9
:107FA000060EDB6A070EDB6A0CD0020EDBCF0FF089
:107FB000030EDBCF10F0060E0FC0DBFF070E10C064
:107FC000DBFF060EDBCF00F0070EDBCF01F000C0B9
:107FD000F3FF01C0F4FF00D0D9CFE1FFE552E7CFB6
:107FE000D9FF1200D9CFE6FFE1CFD9FF080EE12675
:107FF000150EE66E040EE66ECCEC27F0E552E55267
:10800000D9CFE6FFDACFE6FFB0CEE6FFB1CEE6FF8E
:1080100094EC26F0E106E106E106E106D9CFE6FFA1
:10802000DACFE6FF17EC28F0E552E552270EE66EB0
:10803000040EE66ECCEC27F0E552E552D9CFE6FF10
:10804000DACFE6FF0E01B251E66EE66A94EC26F056
:10805000E106E106E106E106D9CFE6FFDACFE6FF69
:1080600017EC28F0E552E5523D0EE66E040EE66E82
:10807000CCEC27F0E552E552D9CFE6FFDACFE6FFA8
:108080000E01A551E66EE66A94EC26F0E106E106E3
:10809000E106E106D9CFE6FFDACFE6FF17EC28F0DC
:1080A000E552E5524E0EE66E040EE66ECCEC27F07D
:1080B000E552E552D9CFE6FFDACFE6FFA6CEE6FFDE
:1080C000A7CEE6FF94EC26F0E106E106E106E10624
:1080D000D9CFE6FFDACFE6FF17EC28F0E552E552FC
:1080E000610EE66E040EE66ECCEC27F0E552E5522A
:1080F000D9CFE6FFDACFE6FFAACEE6FFABCEE6FFAA
:1081000094EC26F0E106E106E106E106D9CFE6FFB0
:10811000DACFE6FF17EC28F0E552E552810EE66E65
:10812000040EE66ECCEC27F0E552E552D9CFE6FF1F
:10813000DACFE6FFA8CEE6FFA9CEE6FF94EC26F064
:10814000E106E106E106E106D9CFE6FFDACFE6FF78
:1081500017EC28F0E552E552000EE66E040EE66ECE
:10816000CCEC27F0E552E552D9CFE6FFDACFE6FFB7
:10817000A3CEE6FFA4CEE6FF94EC26F0E106E106EE
:10818000E106E106D9CFE6FFDACFE6FF17EC28F0EB
:10819000E552E552A10EE66E040EE66ECCEC27F039
:1081A000E552E552D9CFE6FFDACFE6FF0E01A35143
:1081B000B325006EA451B421016E00C0E6FF01C0DA
:1081C000E6FF94EC26F0E106E106E106E106D9CFF0
:1081D000E6FFDACFE6FF17EC28F0E552E552B00EE5
:1081E000E66E040EE66ECCEC27F0E552E552D9CFF0
:1081F000E6FFDACFE6FF0E01A351AA25026EA451D5
:10820000AB21036E0250B325006E0350B421016E02
:1082100000C0E6FF01C0E6FF94EC26F0E106E106AF
:10822000E106E106D9CFE6FFDACFE6FF17EC28F04A
:10823000E552E552730EE66E040EE66ECCEC27F0C6
:10824000E552E552D9CFE6FFDACFE6FFACCEE6FF46
:10825000ADCEE6FF94EC26F0E106E106E106E1068C
:10826000D9CFE6FFDACFE6FF17EC28F0E552E5526A
:10827000930EE66E040EE66ECCEC27F0E552E55266
:10828000D9CFE6FFDACFE6FFAECEE6FFAFCEE6FF10
:1082900094EC26F0E106E106E106E106D9CFE6FF1F
:1082A000DACFE6FF17EC28F0E552E552D9CFE1FF2F
:1082B000E552E7CFD9FF12000E017891796B1200D9
:1082C000D9CFE6FFE1CFD9FF060EE12684A611D073
:1082D0000E0178A10CD078918588B40EE66E010E5F
:1082E000E66ECCEC27F0E552E5529DEC21F0DF6A1A
:1082F000D6D00E0178B1D2D0020EDB6A030EDB6A53
:10830000020EDBCF00F0030EDBCF01F0D00E005CDD
:10831000070E015806E2020EDB2A030E01E3DB2AF8
:10832000EFD70E0178818598A50EE66E010EE66EF8
:10833000CCEC27F0E552E552F29EBCDCF28E0E0149
:10834000B55102E09BEC21F0010EDB6A0101745192
:10835000751125E1200EF36E010EDBCFF4FFF35013
:10836000F45C1DE2010EDB500E01016AAC25006ECB
:10837000AD51012200C0E6FF01C0E6FFC70EE66E68
:10838000010EE66EFFEC4DF0E106E106E106E106C6
:10839000F3CF74F1F4CF75F1010EDB2AD7D7745106
:1083A000751101E07AD0F29EACCEE6FFADCEE6FFCD
:1083B000010EE66E000EE66EE66AC70EE66E010E70
:1083C000E66EC6EC47F0F56E070EE15EF550F28EF4
:1083D000010EDB6A100EF36E010EDBCFF4FFF350DB
:1083E000F45C0BE2010EDB50EA6AB80FE96E0E0E88
:1083F000EA22EF6A010EDB2AEDD7020EDB6A030EDA
:10840000DB6A020EDBCF00F0030EDBCF01F0400E83
:10841000005C000E015816E2100EE66EE66AB80E19
:10842000E66E0E0EE66E000EE66EE66ABEEC4CF0F0
:10843000F56E060EE15EF550020EDB2A030E01E337
:10844000DB2ADFD7010EDB6A01017451751125E1CA
:10845000200EF36E010EDBCFF4FFF350F45C1DE24F
:10846000010EDB500E01016AAC25006EAD510122F8
:1084700000C0E6FF01C0E6FFC70EE66E010EE66E25
:10848000FFEC4DF0E106E106E106E106F3CF74F101
:10849000F4CF75F1010EDB2AD7D700D0DF68DF50AB
:1084A00000D0D9CFE1FFE552E7CFD9FF1200D9CFF5
:1084B000E6FFE1CFD9FF030EE126020EDF6EDB6A95
:1084C000DF50010837E2030EF36E020EDBCFF4FF3C
:1084D000F350F45C2FE2000EE66E060EE66EE66ADE
:1084E000010EE66EFD0EDBCFE6FFFE0EDBCFE6FFF4
:1084F000F3EC34F0F56E060EE15EF550000EE66E1C
:10850000070EE66EE66A010EE66E03EC36F0E10653
:10851000E106E106E10667EC36F0DF6EDF500108A8
:1085200006E24AEC36F0E76E010EE7CFDBFF020E03
:10853000DB2AC6D7D9CFE1FFE552E7CFD9FF12003A
:10854000D9CFE6FFE1CFD9FF030EE126020EDF6EA1
:10855000DB6ADF50010837E2030EF36E020EDBCF59
:10856000F4FFF350F45C2FE2000EE66E060EE66EAA
:10857000E66A010EE66EFD0EDBCFE6FFFE0EDBCFF8
:10858000E6FF92EC36F0F56E060EE15EF550000E59
:10859000E66E070EE66EE66A010EE66EACEC37F0AC
:1085A000E106E106E106E10667EC36F0DF6EDF503A
:1085B000010806E24AEC36F0E76E010EE7CFDBFF7A
:1085C000020EDB2AC6D7D9CFE1FFE552E7CFD9FFAC
:1085D0001200D9CFE6FFE1CFD9FFBF0EE66E010E44
:1085E000E66EC00EE66E010EE66EFD0EDBCF02F00B
:1085F000FE0EDBCF03F00350020AE8AE02D0D890A3
:1086000004D0000E025C020E035802E2000E01D0FC
:10861000010E006E016A00BE016800C0E6FF01C0E5
:10862000E6FFE1EC22F0F56E060EE15EF550FD0E80
:10863000DBCF00F0FE0EDBCF01F00150010AE8AE07
:1086400002D0D89004D0000E005C010E01580CE25C
:10865000FD0EDBCFE9FFFE0EDBCFEAFF000EE926C1
:10866000060EEA22EF5010D0FD0EDBCFE9FFFE0E22
:10867000DBCFEAFF000EE95E010EEA5A000EE926A2
:10868000070EEA22EF5000D0E552E7CFD9FF1200E3
:10869000D9CFE6FFE1CFD9FF020EE126D30EE66E79
:1086A000010EE66EC00EE66E010EE66EFD0EDBCF2D
:1086B00002F0FE0EDBCF03F00350020AE8AE02D058
:1086C000D89004D0000E025C020E035802E2000EA5
:1086D00001D0010E006E016A00BE016800C0E6FF15
:1086E00001C0E6FFE1EC22F0F56E060EE15EF5500A
:1086F000D40EE66E010EE66EC00EE66E010EE66E5C
:10870000010EE76EFD0EDBCF00F0FE0EDBCF01F0B9
:10871000E7500016016A00C0E6FF01C0E6FFE1EC89
:1087200022F0F56E060EE15EF550FD0EDB2AFE0E20
:1087300001E3DB2AFD0EDBCF00F0FE0EDBCF01F004
:108740000150010AE8AE02D0D89004D0000E005CBF
:10875000010E015838E2FD0EDBCFE9FFFE0EDBCF44
:10876000EAFF000EE926060EEA22EF50DE6EDD6A11
:10877000DECF00F0DDCF01F000C001F0006A00C0E4
:10878000DEFF01C0DDFFFD0EDB06FE0E01E2DB06B3
:10879000FD0EDBCFE9FFFE0EDBCFEAFF000EE92680
:1087A000060EEA22EF50E76E000EDFCF00F0010E5A
:1087B000DBCF01F0E7500026000E012200C0DEFFF3
:1087C00001C0DDFF47D0FD0EDBCF00F0FE0EDBCF9A
:1087D00001F0000E005E010E015AFD0E00C0DBFF2D
:1087E000FE0E01C0DBFFFD0EDBCFE9FFFE0EDBCF8F
:1087F000EAFF000EE926070EEA22EF50DE6EDD6A80
:10880000DECF00F0DDCF01F000C001F0006A00C053
:10881000DEFF01C0DDFFFD0EDB06FE0E01E2DB0622
:10882000FD0EDBCFE9FFFE0EDBCFEAFF000EE926EF
:10883000070EEA22EF50E76E000EDFCF00F0010EC8
:10884000DBCF01F0E7500026000E012200C0DEFF62
:1088500001C0DDFFDECF00F0DDCF01F000C0F3FF8F
:1088600001C0F4FF00D0D9CFE1FFE552E7CFD9FF37
:108870001200D9CFE6FFE1CFD9FFED0EE66E010E73
:10888000E66EC00EE66E010EE66EFD0EDBCF02F068
:10889000FE0EDBCF03F00350020AE8AE02D0D89000
:1088A00004D0000E025C020E035802E2000E01D05A
:1088B000010E006E016A00BE016800C0E6FF01C043
:1088C000E6FFE1EC22F0F56E060EE15EF550FD0EDE
:1088D000DBCF00F0FE0EDBCF01F00150010AE8AE65
:1088E00002D0D89004D0000E005C010E01580EE2B8
:1088F000FD0EDBCFE9FFFE0EDBCFEAFF000EE9261F
:10890000060EEA22FC0EDBCFEFFF11D0FD0EDBCF0F
:10891000E9FFFE0EDBCFEAFF000EE95E010EEA5A28
:10892000000EE926070EEA22FC0EDBCFEFFFE55230
:10893000E7CFD9FF1200D9CFE6FFE1CFD9FF020E72
:10894000E126010EE66E020EE66EC00EE66E010E28
:10895000E66EFD0EDBCF02F0FE0EDBCF03F0035020
:10896000020AE8AE02D0D89004D0000E025C020EDB
:10897000035802E2000E01D0010E006E016A00BE33
:10898000016800C0E6FF01C0E6FFE1EC22F0F56EF1
:10899000060EE15EF550020EE66EE66EC00EE66E65
:1089A000010EE66E010EE76EFD0EDBCF00F0FE0E4F
:1089B000DBCF01F0E7500016016A00C0E6FF01C0FE
:1089C000E6FFE1EC22F0F56E060EE15EF550FD0EDD
:1089D000DBCF00F0FE0EDBCF01F00150010AE8AE64
:1089E00002D0D89004D0000E005C010E015834E291
:1089F000FF0EE76EFB0EDBCF00F0FC0EDBCF01F0CD
:108A0000E7500016016AFD0EDBCFE9FFDB2AFE0E00
:108A1000DBCFEAFF01E3DB2A000EE926060EEA229D
:108A200000C0EFFFFB0EDBCF00F0FC0EDBCF01F050
:108A3000000E0016FF0E011601C000F0016AFD0EC7
:108A4000DBCFE9FFFE0EDBCFEAFF000EE926060EC4
:108A5000EA2200C0EFFF3BD0D950FD0FE96EFF0EB8
:108A6000DA20EA6EEE52ED06FF0EE76EFB0EDBCF6C
:108A700000F0FC0EDBCF01F0E7500016016AFD0E9E
:108A8000DBCFE9FFDB2AFE0EDBCFEAFF01E3DB2AC7
:108A9000000EE926070EEA2200C0EFFFFB0EDBCF37
:108AA00000F0FC0EDBCF01F0000E0016FF0E0116E9
:108AB00001C000F0016AFD0EDBCFE9FFFE0EDBCF47
:108AC000EAFF000EE926070EEA2200C0EFFFD9CF29
:108AD000E1FFE552E7CFD9FF1200D9CFE6FFE1CFA2
:108AE000D9FF070EE1260B0EF36E020EF3CFDBFF6C
:108AF000030EDB6ADE68DD68040EDB6A050EDB6AE6
:108B0000020EDBCF00F0030EDBCF01F00150020AB2
:108B1000E8AE02D0D89004D0000E005C020E0158DE
:108B200058E2DECF02F0DDCF03F00001800E031526
:108B300050E0020EDBCFE6FF030EDBCFE6FF49DDA0
:108B4000E552E552E76E060EE7CFDBFFDB500F087C
:108B500031E0D950020FE96EDACFEAFF0B0EEE5E7C
:108B6000000EED5A020EDBCFE6FF030EDBCFE6FF71
:108B700030DDE552E552E76E060EE7CFDBFFDB5056
:108B800004E0060EDB50E50806E1040EDBCFDEFF55
:108B9000DBCFDDFF0ED0D950020FE96EDACFEAFF4E
:108BA0002B0EEE26000EED22040EDB2A050E01E34D
:108BB000DB2A0ED0D950020FE96EDACFEAFF200E81
:108BC000EE26000EED22040EDB2A050E01E3DB2A61
:108BD00097D7DECF00F0DDCF01F000C0F3FF01C07A
:108BE000F4FF00D0D9CFE1FFE552E7CFD9FF120063
:108BF000D9CFE6FFE1CFD9FF040EE12681EC38F0B2
:108C0000DDEC38F00001BF390F0B0A0DF350DE6EBA
:108C1000DD6A0F0EBF15DE26000EDD22D9CFE9FF7B
:108C2000DACFEAFF020EEECFDBFF030EEDCFDBFF64
:108C3000D950020FE96EDACFEAFF0B0ED890EE366C
:108C4000ED36E806FBE10001BE390F0B0A0DF350CB
:108C5000DE6EDD6A0F0EBE15DE26000EDD22DECFD3
:108C600000F0DDCF01F0050ED89000360136E804A3
:108C7000FBE1D950020FE96EDACFEAFF0050EE2691
:108C80000150ED22020EDBCF00F0030EDBCF01F02E
:108C900000C0F3FF01C0F4FF00D0D9CFE1FFE552DF
:108CA000E7CFD9FF1200D9CFE6FFE1CFD9FF040EFD
:108CB000E12681EC38F0DDEC38F00001C3390F0B10
:108CC0000A0DF350DE6EDD6A0F0EC315DE26000EB0
:108CD000DD22140EDE26000EDD22DECF00F0DDCF19
:108CE00001F000C001F0006AD8900136020E00C009
:108CF000DBFF030E01C0DBFFC2390F0B010B0A0DB6
:108D0000F350DE6EDD6A0F0EC215DE26000EDD2288
:108D1000DECF00F0DDCF01F0050ED8900036013631
:108D2000E804FBE1D950020FE96EDACFEAFF005008
:108D3000EE260150ED220001C1390F0B0A0DF35050
:108D4000DE6EDD6A0F0EC115DE26000EDD22DECFDF
:108D500000F0DDCF01F0D950020FE96EDACFEAFF63
:108D60000050EE260150ED22020EDBCF00F0030E84
:108D7000DBCF01F000C0F3FF01C0F4FF00D0D9CF7A
:108D8000E1FFE552E7CFD9FF1200D9CFE6FFE1CFEF
:108D9000D9FF070EE126000E0E018415006EFF0EAE
:108DA0008515016E050E00C0DBFF060E01C0DBFF5E
:108DB000D950050FE96EDACFEAFF040E0F0B06E07B
:108DC000EC52D890ED32EF32E806FAE1D950050FB7
:108DD000E96EDACFEAFF040E0F0B06E0EC52D890F2
:108DE000ED32EF32E806FAE1D950050FE96EDACF3D
:108DF000EAFF0E01B351EE26B451ED22050EDB5011
:108E0000A3250001006F060EDB500E01A421000116
:108E1000016F00C0E6FF01C0E6FF57EC42F0E552EB
:108E2000E552040EDE6EDD6ADECFE6FFDDCFE6FF43
:108E30002FDCE552E552020EF3CFDBFF030EF4CF39
:108E4000DBFF040EDB6AD950020FE96EDACFEAFFCE
:108E5000EE50ED1059E0040EDB5056E1020EDE2616
:108E6000000EDD22DECF00F0DDCF01F0005C020E4F
:108E700001580FE2DECFE6FFDDCFE6FF48EC43F01E
:108E8000E552E552020EF3CFDBFF030EF4CFDBFF1A
:108E90003AD0050EDBCF00F0060EDBCF01F00E015D
:108EA0000050AA5D0150AB5929E3050EDB2A060EDE
:108EB00001E3DB2A050EDB50A3250001006F060E3F
:108EC000DB500E01A4210001016F00C0E6FF01C0CC
:108ED000E6FF57EC42F0E552E552DE6ADD6ADECF8E
:108EE000E6FFDDCFE6FF48EC43F0E552E552020E27
:108EF000F3CFDBFF030EF4CFDBFF05D0010EF36EE3
:108F0000040EF3CFDBFF9FD7040EDB5036E1050ED6
:108F1000DBCF00F0060EDBCF01F00006000E015A99
:108F2000040ED89000360136E804FBE1FD0EDBCFDD
:108F3000E9FFFE0EDBCFEAFF00C0EEFF01C0EDFF50
:108F4000FD0EDBCFE9FFFE0EDBCFEAFF040ED8906B
:108F5000EE36ED36E806FBE1DECF00F0DDCF01F0C6
:108F6000D89001320032FD0EDBCFE9FFFE0EDBCFE1
:108F7000EAFF0050EE260150ED22040EDB5000D037
:108F8000D9CFE1FFE552E7CFD9FF1200D9CFE6FFF5
:108F9000E1CFD9FF0F0EE12660EC41F0000901E1BD
:108FA0004DD20E01B55101E143D2020EDB6A030E30
:108FB000DB68040EDB68F80EDBCF00F0F90EDBCFC8
:108FC00001F0AC51001802E1AD51011838E1020E78
:108FD000DBCF00F00E01A851005C000EA9552EE277
:108FE000030EDBCF01F0040EDBCF02F00001800E98
:108FF000021524E0020EDB500E01016AAC25006E62
:10900000AD51012200C0E6FF01C0E6FF57EC42F07F
:10901000E552E55262DD030EF3CFDBFF040EF4CF21
:10902000DBFF030EDBCF00F0040EDBCF01F000010D
:10903000800E011502E0020EDB2AC9D711D0F80E0E
:10904000DBCFE6FFF90EDBCFE6FF57EC42F0E5524F
:10905000E55243DD030EF3CFDBFF040EF4CFDBFF5D
:10906000030EDBCF00F0040EDBCF01F00001800E19
:10907000011501E0D6D1020EDB500E017A6F7B6B39
:10908000030EDBCF7CFE040EDBCF7DFE826B836B99
:10909000846B856B7E6B7F6B806B816B200E0F6E9C
:1090A000106A030EDBCF14F0040EDBCF15F000ECDA
:1090B00026F0070E0DC0DBFF080E0EC0DBFF050E0D
:1090C000DB6A060EDB6AFD0EDBCFE9FFFE0EDBCFAF
:1090D000EAFFEF502CE0FD0EDBCFE9FFFE0EDBCF09
:1090E000EAFFEF502E0823E0FD0EDBCFE9FFFE0E76
:1090F000DBCFEAFFEF50E66E070EDBCFE6FF080E90
:10910000DBCFE6FF39EC44F0E106E106E106070EAD
:10911000DB2A080E01E3DB2AFD0EDB2AFE0E01E34B
:10912000DB2A050EDB2A060E01E3DB2ACCD7050E6F
:10913000DBCF00F0060EDBCF01F0080E005C000E66
:10914000015818E2200EE66E070EDBCFE6FF080E90
:10915000DBCFE6FF39EC44F0E106E106E106070E5D
:10916000DB2A080E01E3DB2A050EDB2A060E01E3EB
:10917000DB2ADDD7FD0EDBCFE9FFFE0EDBCFEAFFFA
:10918000EF502E0862E1FD0EDB2AFE0E01E3DB2A22
:10919000050EDB6A060EDB6AFD0EDBCFE9FFFE0E75
:1091A000DBCFEAFFEF502EE0050EDBCF00F0060E1E
:1091B000DBCF01F0030E005C000E015823E2FD0E30
:1091C000DBCFE9FFFE0EDBCFEAFFEF50E66E070EC6
:1091D000DBCFE6FF080EDBCFE6FF39EC44F0E1061B
:1091E000E106E106070EDB2A080E01E3DB2AFD0E8D
:1091F000DB2AFE0E01E3DB2A050EDB2A060E01E365
:10920000DB2ACAD7050EDBCF00F0060EDBCF01F05C
:10921000030E005C000E015818E2200EE66E070EE9
:10922000DBCFE6FF080EDBCFE6FF39EC44F0E106CA
:10923000E106E106070EDB2A080E01E3DB2A050E34
:10924000DB2A060E01E3DB2ADDD7FA0EDB5000082D
:1092500013E2100EE66E070EDBCFE6FF080EDBCF43
:10926000E6FF39EC44F0E106E106E106070EDB2AF1
:10927000080E01E3DB2A11D0E66A070EDBCFE6FF1A
:10928000080EDBCFE6FF39EC44F0E106E106E1062B
:10929000070EDB2A080E01E3DB2A050EDB6A060E49
:1092A000DB6A050EDBCF00F0060EDBCF01F00A0E05
:1092B000005C000E015817E2E66A070EDBCFE6FFFE
:1092C000080EDBCFE6FF39EC44F0E106E106E106EB
:1092D000070EDB2A080E01E3DB2A050EDB2A060E49
:1092E00001E3DB2ADED784DC090EF3CFDBFF0A0EB5
:1092F000F4CFDBFF090EDBCFE6FF0A0EDBCFE6FF84
:10930000070EDBCFE6FF080EDBCFE6FF9BEC44F059
:10931000E106E106E106E106D950070FE96EDACF72
:10932000EAFF020EEE26000EED22BDDC090EF3CFA1
:10933000DBFF0A0EF4CFDBFF090EDBCFE6FF0A0EE0
:10934000DBCFE6FF070EDBCFE6FF080EDBCFE6FF45
:109350009BEC44F0E106E106E106E106D950070F77
:10936000E96EDACFEAFF020EEE26000EED22050EC0
:10937000DB6A060EDB6A050EDBCF00F0060EDBCFE4
:1093800001F0005C000E015817E2E66A070EDBCF21
:10939000E6FF080EDBCFE6FF39EC44F0E106E1061C
:1093A000E106070EDB2A080E01E3DB2A050EDB2AA5
:1093B000060E01E3DB2ADFD7F80EDBCF00F0F90E53
:1093C000DBCF01F00E01AC51001802E1AD510118E4
:1093D00010E1020EDB50016AAC25006EAD51012296
:1093E00000C0E6FF01C0E6FFA0EC42F0E552E55206
:1093F0000AD0F80EDBCFE6FFF90EDBCFE6FFA0ECDC
:1094000042F0E552E552F80EDBCF8BFEF90EDBCFD2
:109410008CFE0E01010E796FDE6ADD6AB66BB76BEA
:1094200006D0DE68DD680E019A0EB66FB76905D00A
:10943000DE68DD689B0EB66FB76906D0DE68DD6852
:109440000E019C0EB66FB769DECF00F0DDCF01F0E4
:1094500000C0F3FF01C0F4FF00D0D9CFE1FFE55217
:10946000E7CFD9FF1200D9CFE6FFE1CFD9FF020E37
:10947000E1260E01000ED8808455000E855501E3CB
:10948000DED0000E8415046EFF0E8515056E05C036
:1094900004F0056AA3510424026EA4510520036E52
:1094A0000250B325006E0350B421016E00C0DEFFF0
:1094B00001C0DDFFDECFE6FFDDCFE6FF57EC42F077
:1094C000E552E552E668E668FF0E0E018415006E6F
:1094D000016AD8900036013600C0E6FF01C0E6FF01
:1094E0009BEC44F0E106E106E106E106DECFE6FF93
:1094F000DDCFE6FFA0EC42F0E552E552DE500E0172
:10950000AA250001006FDD500E01AB210001016FA3
:1095100000C0E6FF01C0E6FFA0EC42F0E552E552D4
:109520000E01825183113AE18B517A25006E8C51E4
:109530007B21016E00C0E6FF01C0E6FF57EC42F060
:10954000E552E55284CEE6FF85CEE6FF7CCE00F004
:109550007DCE01F0050ED89000360136E806FBE11D
:109560001A0E0026000E012200C0E6FF01C0E6FF31
:109570009BEC44F0E106E106E106E1060E018B51A9
:109580007A25006E8C517B21016E00C0E6FF01C080
:10959000E6FFA0EC42F0E552E55251D0000E8215F4
:1095A000046EFF0E8315056E05C004F0056AA35115
:1095B0000424026EA4510520036E0250B325006EF0
:1095C0000350B421016E00C0DEFF01C0DDFFDECF1D
:1095D000E6FFDDCFE6FF57EC42F0E552E55284CEE0
:1095E000E6FF85CEE6FFFF0E0E018215006E016AD2
:1095F000D8900036013600C0E6FF01C0E6FF9BECC4
:1096000044F0E106E106E106E106DECFE6FFDDCF4C
:10961000E6FFA0EC42F0E552E552DE500E01AA252D
:109620000001006FDD500E01AB210001016F00C091
:10963000E6FF01C0E6FFA0EC42F0E552E552D9CFCB
:10964000E1FFE552E7CFD9FF1200D9CFE6FFE1CF26
:10965000D9FF060EE1260E018B517A25006E8C5142
:109660007B21016E00C0E6FF01C0E6FF57EC42F02F
:10967000E552E5527CCE04F07DCE05F0050ED89083
:1096800004360536E806FBE11E0E0426000E052210
:1096900004C0E6FF05C0E6FF48EC43F0E552E552A2
:1096A000F3CF00F0F4CF01F0026A036A00C0DFFFDD
:1096B000010E01C0DBFF020E02C0DBFF030E03C080
:1096C000DBFFD9CFE9FFDACFEAFF040EE76ED890CF
:1096D000000EEF36010EEB36020EEB36030EEB36C4
:1096E000E706F5E1D9CFE9FFDACFEAFF040EE76E2E
:1096F000D890000EEF36010EEB36020EEB36030E5D
:10970000EB36E706F5E1D9CFE9FFDACFEAFF040E41
:10971000E76ED890000EEF36010EEB36020EEB36F8
:10972000030EEB36E706F5E1D9CFE9FFDACFEAFF22
:10973000040EE76ED890000EEF36010EEB36020EE7
:10974000EB36030EEB36E706F5E17CCE00F07DCE7E
:1097500001F0050ED89000360136E806FBE11C0E3C
:109760000026000E012200C0E6FF01C0E6FF48EC23
:1097700043F0E552E552040EF3CFDBFF050EF4CFC4
:10978000DBFF040EDBCF04F0050EDBCF05F0066A2D
:10979000076AD9CFE9FFDACFEAFFEE500424006E62
:1097A000EE500520016EEE500620026EEE500720AE
:1097B000036E00C0DFFF010E01C0DBFF020E02C01E
:1097C000DBFF030E03C0DBFFFD0EDBCF04F0FE0E5C
:1097D000DBCF05F0066A076AD9CFE9FFDACFEAFFE7
:1097E000EE500424006EEE500520016EEE5006206F
:1097F000026EEE500720036E00C0DFFF010E01C0B5
:10980000DBFF020E02C0DBFF030E03C0DBFFD9CF7C
:10981000E9FFDACFEAFFEECF00F0EECF01F0EECFB6
:1098200002F0EFCF03F0026A036A040E00C0DBFF10
:10983000050E01C0DBFF040EDBCFE6FF050EDBCF1C
:10984000E6FF7CCE00F07DCE01F0D89000360136E8
:10985000E806FBE11C0E0026000E012200C0E6FF18
:1098600001C0E6FF9BEC44F0E106E106E106E106FB
:10987000D9CFE9FFDACFEAFF040EE76ED890030EE6
:10988000EB32020EEB32010EEB32EF32E706F6E17D
:10989000D9CFE9FFDACFEAFF040EE76ED890030EC6
:1098A000EB32020EEB32010EEB32EF32E706F6E15D
:1098B000D9CFE9FFDACFEAFF040EE76ED890030EA6
:1098C000EB32020EEB32010EEB32EF32E706F6E13D
:1098D000D9CFE9FFDACFEAFF040EE76ED890030E86
:1098E000EB32020EEB32010EEB32EF32E706F6E11D
:1098F000D9CFE9FFDACFEAFFEECF00F0EECF01F0EB
:10990000EECF02F0EFCF03F0026A036A040E00C04C
:10991000DBFF050E01C0DBFF040EDBCFE6FF050E0B
:10992000DBCFE6FF7CCE00F07DCE01F0D890003694
:109930000136E806FBE11E0E0026000E012200C0E3
:10994000E6FF01C0E6FF9BEC44F0E106E106E1061C
:10995000E1060E018B517A25006E8C517B21016E40
:1099600000C0E6FF01C0E6FFA0EC42F0E552E55280
:10997000D9CFE1FFE552E7CFD9FF1200D9CFE6FFFB
:10998000E1CFD9FF040EE126DE6ADD6A0E0179051A
:1099900001E010D18451851115E1840EE66E0E0EA2
:1099A000E66EC5EC46F0E552E552000807E2DE68D7
:1099B000DD680E01990EB66FB76904D00E01866B93
:1099C000876B886BDECF00F0DDCF01F00001800EE9
:1099D000011501E0D9D00E01B251046E056A84CEA2
:1099E00002F085CE03F0020E025E000E035A02C0A2
:1099F0000FF003C010F004C014F005C015F02DECFA
:109A000026F00D500E01AE25006E0E50AF21016EF6
:109A100086518A6B0024896F01508A2389CEE6FF24
:109A20008ACEE6FF57EC42F0E552E552F90EDBCF65
:109A30000FF0FA0EDBCF10F0020E0FC0DBFF030EAB
:109A400010C0DBFFD950020FE96EDACFEAFFEE500B
:109A5000ED1001E181D00E01000E875D020E8859E4
:109A60005BE389CEE6FF8ACEE6FFA0EC42F0E5524A
:109A7000E5520E01862BB251865D06E2892B000E5F
:109A80008A23876B886B47D0840EE66E0E0EE66ED7
:109A9000C5EC46F0E552E552000817E2020EDB6A1B
:109AA000030EDB6A020EDBCF0FF0030EDBCF10F0EC
:109AB000F90E0FC0DBFFFA0E10C0DBFFDE68DD68B9
:109AC0000E01990EB66FB76926D00E01866B876BB3
:109AD000886BB251046E056A84CE02F085CE03F025
:109AE000020E025E000E035A02C00FF003C010F017
:109AF00004C014F005C015F02DEC26F00D500E0139
:109B0000AE25006E0E50AF21016E86518A6B002487
:109B1000896F01508A231FD0FB0EDBCFE9FFFC0EBB
:109B2000DBCFEAFFEF50E66E87CEE6FF88CEE6FF9A
:109B300039EC44F0E106E106E1060E01872B000E48
:109B40008823FB0EDB2AFC0E01E3DB2A020EDB0678
:109B5000030E01E2DB0676D70E01000E875D020ED2
:109B600088590AE2E66A87CEE6FF88CEE6FF39EC3E
:109B700044F0E106E106E10689CEE6FF8ACEE6FF83
:109B8000A0EC42F0E552E5520E018451821902E147
:109B90008551831905E067DC84CE82FE85CE83FE85
:109BA000F90EDBCFE6FFFA0EDBCFE6FF4EDDE55226
:109BB000E55205D0DE68DD68380EB66FB769DECFD6
:109BC00000F0DDCF01F000C0F3FF01C0F4FF00D0D2
:109BD000D9CFE1FFE552E7CFD9FF1200D9CFE6FF99
:109BE000E1CFD9FF020EE126DE6ADD6A0E01796B54
:109BF00000D0D9CFE1FFE552E7CFD9FF1200D9CF8E
:109C0000E6FFE1CFD9FF090EE126030EDB6A040E61
:109C1000DB6A070EDB6AFB0EDBCFE6FFFC0EDBCF59
:109C2000E6FF57EC42F0E552E552DF6A010EDB6ACF
:109C3000020EDB6A010EDBCF00F0020EDBCF01F07B
:109C4000FF0E005C000E01583AE2070EDB0437E01D
:109C5000010EDBCFE9FF020EDBCFEAFF000EE926A3
:109C6000060EEA22EFCF00F0DF50E76EFD0EDBCFED
:109C7000E9FFFE0EDBCFEAFFE750E926000EEA22FD
:109C8000EF50005C15E1010EDB2A020E01E3DB2A36
:109C9000DF2A0A0EDF5C0BE1010EF36E070EF3CF35
:109CA000DBFF010EDB50E76E080EE7CFDBFFD0D7FE
:109CB000DF6A010EDB2A020E01E3DB2ABBD7070EA7
:109CC000DB5001E0BCD0DF6A010EDB6A020EDB6A0A
:109CD000010EDBCF00F0020EDBCF01F0FF0E005CC7
:109CE000000E01583AE2070EDB0437E0010EDBCF2D
:109CF000E9FF020EDBCFEAFF000EE926070EEA229B
:109D0000EFCF00F0DF50E76EFD0EDBCFE9FFFE0E78
:109D1000DBCFEAFFE750E926000EEA22EF50005CB5
:109D200015E1010EDB2A020E01E3DB2ADF2A0A0E0F
:109D3000DF5C0BE1010EF36E070EF3CFDBFF010ECC
:109D4000DB50E76E080EE7CFDBFFD0D7DF6A010EEE
:109D5000DB2A020E01E3DB2ABBD7070EDB506EE0E5
:109D6000080EDB50110FEA6A000FE96E070EEA22B7
:109D7000EF50E66ED950030FE96EDACFEAFFE552F5
:109D8000E750EE6EED6A030EDBCF00F0040EDBCF82
:109D900001F000C001F0006A050E00C0DBFF060EF6
:109DA00001C0DBFF080EDB50100FEA6A000FE96EFE
:109DB000070EEA22EF50E66ED950030FE96EDACFB4
:109DC000EAFFE552E750EE6EED6A050EDBCF00F0DC
:109DD000060EDBCF01F0D950030FE96EDACFEAFFB0
:109DE0000050EE260150ED22D950030FE96EDACF74
:109DF000EAFF020EEE5E000EED5A0E01B251006E49
:109E0000016AD950030FE96EDACFEAFF00C014F0FF
:109E100001C015F0EECF0FF0EDCF10F02DEC26F0D5
:109E20000DC0EEFF0EC0EDFFD950030FE96EDACF83
:109E3000EAFF0E01AE51EE26AF51ED226ED0080EB4
:109E4000DB50110FEA6A000FE96E060EEA22EF50AE
:109E5000E66ED950030FE96EDACFEAFFE552E7501C
:109E6000EE6EED6A030EDBCF00F0040EDBCF01F0E7
:109E700000C001F0006A050E00C0DBFF060E01C045
:109E8000DBFF080EDB50100FEA6A000FE96E060ECA
:109E9000EA22EF50E66ED950030FE96EDACFEAFFFF
:109EA000E552E750EE6EED6A050EDBCF00F0060ED0
:109EB000DBCF01F0D950030FE96EDACFEAFF005093
:109EC000EE260150ED22D950030FE96EDACFEAFFFA
:109ED000020EEE5E000EED5A0E01B251006E016AE6
:109EE000D950030FE96EDACFEAFF00C014F001C0C9
:109EF00015F0EECF0FF0EDCF10F02DEC26F00DC0E9
:109F0000EEFF0EC0EDFFD950030FE96EDACFEAFF86
:109F10000E01AE51EE26AF51ED22030EDBCF00F065
:109F2000040EDBCF01F000C0F3FF01C0F4FF00D04E
:109F3000D9CFE1FFE552E7CFD9FF1200D9CFE6FF35
:109F4000E1CFD9FF0E0EE1260A0EDB6A0B0EDB6AAB
:109F5000DE68DD68FD0EDBCFE6FFFE0EDBCFE6FF41
:109F600057EC42F0E552E5526DEC45F0F3CFDEFFE1
:109F7000F4CFDDFFDECF00F0DDCF01F00001800E79
:109F8000011501E16FD10E01B251046E056AFD0E9B
:109F9000DBCF0FF0FE0EDBCF10F0AE510F5C026E88
:109FA000AF511058036E02C00FF003C010F004C090
:109FB00014F005C015F0B1EC21F00FC000F010C096
:109FC00001F0020E0026000E01220C0E00C0DBFF85
:109FD0000D0E01C0DBFF0A0EDB6A0B0EDB6A0E0101
:109FE000B251046E056AFD0EDBCF0FF0FE0EDBCF23
:109FF00010F0AE510F5C026EAF511058036E02C0EC
:10A000000FF003C010F004C014F005C015F0B1EC5F
:10A0100021F00FC000F010C001F0020E0026000E6B
:10A020000122040E00C0DBFF050E01C0DBFFDECF06
:10A0300000F0DDCF01F00001800E011501E178D0C4
:10A04000D950080FE96EDACFEAFF000ED880EE543F
:10A05000000EED546DE2040EDBCFE6FF050EDBCF04
:10A06000E6FF1AEC3FF0E552E552080EF3CFDBFFB6
:10A07000090EF4CFDBFFD950080FE96EDACFEAFF03
:10A08000000ED880EE54000EED5451E20E01B25194
:10A09000046E056A080EDBCF02F0090EDBCF03F079
:10A0A000020E025E000E035A02C00FF003C010F051
:10A0B00004C014F005C015F02DEC26F00D500E0173
:10A0C000AE25006E0E50AF21016E00C0E6FF01C04C
:10A0D000E6FF57EC42F0E552E5526DEC45F0F3CF68
:10A0E000DEFFF4CFDDFF080EDBCF0FF0090EDBCF74
:10A0F00010F00C0E0FC0DBFF0D0E10C0DBFF040EC6
:10A10000DBCF0FF0050EDBCF10F00A0E0FC0DBFF28
:10A110000B0E10C0DBFF080EDBCF0FF0090EDBCFFC
:10A1200010F0040E0FC0DBFF050E10C0DBFF7FD761
:10A13000DECF00F0DDCF01F0800E01156DE00C0EDA
:10A14000DBCF84FE0D0EDBCF85FE0C0EDBCF82FE57
:10A150000D0EDBCF83FEACCE8BFEADCE8CFE0E01A2
:10A16000010E796F866B876B020E886F060EDB6AB5
:10A17000100EF36E060EDBCFF4FFF350F45C0BE22F
:10A18000060EDB50EA6AB80FE96E0E0EEA22EF6A9D
:10A19000060EDB2AEDD7070EDB6A200EF36E070EE4
:10A1A000DBCFF4FFF350F45C13E2100EE66EE66AC8
:10A1B000B80EE66E0E0EE66E000EE66EE66ABEECB9
:10A1C0004CF0F56E060EE15EF550070EDB2AE5D782
:10A1D0000E01B251046E056A82CE02F083CE03F006
:10A1E000020E025E000E035A02C00FF003C010F010
:10A1F00004C014F005C015F02DEC26F00D500E0132
:10A20000AE25006E0E50AF21016E020E00C0DBFFC6
:10A21000030E01C0DBFF25D00E01B251046E056AAA
:10A22000080EDBCF02F0090EDBCF03F0020E025E58
:10A23000000E035A02C00FF003C010F004C014F067
:10A2400005C015F02DEC26F00D500E01AE25006E68
:10A250000E50AF21016E020E00C0DBFF030E01C0E5
:10A26000DBFF0CD0FD0EDBCF0FF0FE0EDBCF10F0CE
:10A27000020E0FC0DBFF030E10C0DBFF020EDBCFB0
:10A2800000F0030EDBCF01F000C0F3FF01C0F4FFCC
:10A2900000D0D9CFE1FFE552E7CFD9FF1200D9CFE7
:10A2A000E6FFE1CFD9FF060EE1260E0178A158D0D6
:10A2B000FD0EDBCFE6FFFE0EDBCFE6FF9EEC58F097
:10A2C000E552E552E76E050EE7CFDBFFDB5036E1E6
:10A2D00074C1E6FF75C1E6FF31DEE552E552020EBC
:10A2E000F3CFDBFF030EF4CFDBFF020EDBCF00F07A
:10A2F000030EDBCF01F00E01AE51005CAF510158EF
:10A300001CE3F29E020EDBCFE6FF030EDBCFE6FF7F
:10A31000E66A000EE66EE66AFD0EDBCFE6FFFE0E95
:10A32000DBCFE6FFC6EC47F0F56E070EE15EF550B9
:10A33000F3CFDEFFF4CFDDFFF28E05D0010EF36E1A
:10A34000040EF3CFDBFFD9CFE9FFDACFEAFFEE50FF
:10A35000ED1005E1010EF36E040EF3CFDBFF02D02A
:10A36000040EDB6A040EDB5000D0D9CFE1FFE552CA
:10A37000E7CFD9FF1200D9CFE6FFE1CFD9FF1B0EFF
:10A38000E126530EDF6EDE52590EDD6E530EF36E74
:10A39000020EF3CFDBFF540EF36E030EF3CFDBFFA1
:10A3A000450EF36E040EF3CFDBFF4D0EF36E050E7C
:10A3B000F3CFDBFF200EF36E060EF3CFDBFF200E94
:10A3C000F36E070EF3CFDBFF200EF36E080EF3CF14
:10A3D000DBFF200EF36E090EF3CFDBFF200EF36ED2
:10A3E0000A0EF3CFDBFF440EF36E0B0EF3CFDBFF51
:10A3F000450EF36E0C0EF3CFDBFF4D0EF36E0D0E1C
:10A40000F3CFDBFF4F0EF36E0E0EF3CFDBFF5F0ECD
:10A41000F36E0F0EF3CFDBFF490EF36E100EF3CF8A
:10A42000DBFF4E0EF36E110EF3CFDBFF490EF36E22
:10A43000120EF3CFDBFF540EF36E130EF3CFDBFFE0
:10A44000580EF36E140EF3CFDBFF540EF36E150EA1
:10A45000F3CFDBFF160EDB6A170EDB6A180EDB6A22
:10A46000190EDB6A1A0EDB6AD950170FE96EDACFC4
:10A47000EAFFEE50ED1027E1200EF36E160EDBCF53
:10A48000F4FFF350F45C1FE2160EDB500E01016A7C
:10A49000AC25006EAD51012200C0E6FF01C0E6FF11
:10A4A000D9CFE6FFDACFE6FFFFEC4DF0E106E1069B
:10A4B000E106E106170EF3CFDBFF180EF4CFDBFF4A
:10A4C000160EDB2AD1D7170EDBCFE6FF180EDBCF37
:10A4D000E6FFD9500B0FE66EDACFE6FFFFEC4DF04A
:10A4E000E106E106E106E106190EF3CFDBFF1A0EE5
:10A4F000F4CFDBFFD950190FE96EDACFEAFFEE5047
:10A50000ED1001E128D2190EDBCFE6FF1A0EDBCFEA
:10A51000E6FF57EC42F0E552E552160EDB6ADB50DF
:10A52000EA6A000FE96E060EEA22EF503D0803E0EA
:10A53000160EDB2AF4D7160EDB2ADB50EA6A000F70
:10A54000E96E060EEA22EF50D00F01016C6F160E75
:10A55000DB50EA6A000FE96E060EEA22EF503D0872
:10A5600003E0160EDB2AF3D7160EDB2A01016B6B14
:10A57000DB50EA6A000FE96E060EEA22EFCF00F028
:10A58000300E005C1BE3160EDB50EA6A000FE96E2A
:10A59000060EEA22EF50390811E30A0E6B03F3CFDF
:10A5A0006BF1160EDB50EA6A000FE96E060EEA2226
:10A5B000EF50D00F6B27160EDB2ADAD7160EDB50C2
:10A5C000EA6A000FE96E060EEA22EF503D0803E04A
:10A5D000160EDB2AF3D7160EDB2A01016D6B6E6BAC
:10A5E0006F6B706BDB50EA6A000FE96E060EEA22B1
:10A5F000EFCF00F0300E005C36E3160EDB50EA6A57
:10A60000000FE96E060EEA22EF5039082CE30A0E1D
:10A61000126E136A146A156A6DC10DF06EC10EF0E8
:10A620006FC10FF070C110F040EC22F009C06DF165
:10A630000AC06EF10BC06FF10CC070F1160EDB504A
:10A64000EA6A000FE96E060EEA22EF50D00F006EA4
:10A650000001005101016D27000E6E236F2370234E
:10A66000160EDB2ABFD7160EDB50EA6A000FE96E22
:10A67000060EEA22EF503D0803E0160EDB2AF3D760
:10A68000160EDB2A0101676BDB50EA6A000FE96EE8
:10A69000060EEA22EFCF00F0300E005C1BE3160E30
:10A6A000DB50EA6A000FE96E060EEA22EF50390825
:10A6B00011E30A0E6703F3CF67F1160EDB50EA6A67
:10A6C000000FE96E060EEA22EF50D00F6727160E34
:10A6D000DB2ADAD7160EDB50EA6A000FE96E060EA7
:10A6E000EA22EF503D0803E0160EDB2AF3D7160EE0
:10A6F000DB2A0101686BDB50EA6A000FE96E060E87
:10A70000EA22EFCF00F0300E005C1BE3160EDB50A8
:10A71000EA6A000FE96E060EEA22EF50390811E3EB
:10A720000A0E6803F3CF68F1160EDB50EA6A000FD9
:10A73000E96E060EEA22EF50D00F6827160EDB2ACC
:10A74000DAD7160EDB50EA6A000FE96E060EEA222F
:10A75000EF503D0803E0160EDB2AF3D7160EDB2A76
:10A7600001016A6BDB50EA6A000FE96E060EEA220D
:10A77000EFCF00F0300E005C1BE3160EDB50EA6AF0
:10A78000000FE96E060EEA22EF50390811E30A0EB7
:10A790006A03F3CF6AF1160EDB50EA6A000FE96E26
:10A7A000060EEA22EF50D00F6A27160EDB2ADAD700
:10A7B000160EDB50EA6A000FE96E060EEA22EF5031
:10A7C0003D0803E0160EDB2AF3D7160EDB2A010143
:10A7D000696BDB50EA6A000FE96E060EEA22EFCFE2
:10A7E00000F0300E005C1BE3160EDB50EA6A000F2F
:10A7F000E96E060EEA22EF50390811E30A0E6903EA
:10A80000F3CF69F1160EDB50EA6A000FE96E060E0F
:10A81000EA22EF50D00F6927160EDB2ADAD7160E80
:10A82000DB50EA6A000FE96E060EEA22EF503D089F
:10A8300003E0160EDB2AF3D7160EDB2A0101716B3B
:10A84000726BDB50EA6A000FE96E060EEA22EFCF68
:10A8500000F0300E005C25E3160EDB50EA6A000FB4
:10A86000E96E060EEA22EF5039081BE30A0E720366
:10A87000F3CF72F17103F3CF71F1F4507227160E1A
:10A88000DB50EA6A000FE96E060EEA22EF50D00FA5
:10A89000006E016A0050712701507223160EDB2AE8
:10A8A000D0D771C100F072C101F0026A000E021827
:10A8B000E8AE02D0023407D09C0ED8800054950E2A
:10A8C0000154000E025403E20B0E716F726B9C0E6A
:10A8D000D88071554A0E725503E2170E716F726B74
:10A8E0001C0ED8807155250E725503E22F0E716F24
:10A8F000726B5C0ED8807155120E725503E25F0EBA
:10A90000716F726BFC0ED8807155080E725503E2A0
:10A91000BF0E716F726B160EDB50EA6A000FE96EA4
:10A92000060EEA22EF503D0803E0160EDB2AF3D7AD
:10A93000160EDB2ADB2ADB2A0101736BDB50EA6A85
:10A94000000FE96E060EEA22EF50040803E1010E43
:10A95000736F01D0736BD9CFE1FFE552E7CFD9FF19
:10A960001200D9CFE6FFE1CFD9FF1E0EE126030E7C
:10A97000DB6A040EDB6A070EDB6A0C0EDB6A0D0E67
:10A98000DB6A0E0EDB6A0F0EDB6A120EDB6A130E39
:10A99000DB6AFB0EDBCFE6FFFC0EDBCFE6FF57ECFE
:10A9A00042F0E552E552DF6A010EDB6A020EDB6A15
:10A9B000010EDBCF00F0020EDBCF01F0FF0E005CDA
:10A9C000000E01583AE2070EDB0437E0010EDBCF40
:10A9D000E9FF020EDBCFEAFF000EE926060EEA22AF
:10A9E000EFCF00F0DF50E76EFD0EDBCFE9FFFE0E8C
:10A9F000DBCFEAFFE750E926000EEA22EF50005CC9
:10AA000015E1010EDB2A020E01E3DB2ADF2A0A0E22
:10AA1000DF5C0BE1010EF36E070EF3CFDBFF010EDF
:10AA2000DB50E76E080EE7CFDBFFD0D7DF6A010E01
:10AA3000DB2A020E01E3DB2ABBD7070EDB5001E065
:10AA400058D1DF6A010EDB6A020EDB6A010EDBCF32
:10AA500000F0020EDBCF01F0FF0E005C000E01588B
:10AA60003AE2070EDB0437E0010EDBCFE9FF020E0E
:10AA7000DBCFEAFF000EE926070EEA22EFCF00F057
:10AA8000DF50E76EFD0EDBCFE9FFFE0EDBCFEAFF06
:10AA9000E750E926000EEA22EF50005C15E1010EB6
:10AAA000DB2A020E01E3DB2ADF2A0A0EDF5C0BE160
:10AAB000010EF36E070EF3CFDBFF010EDB50E76EE6
:10AAC000080EE7CFDBFFD0D7DF6A010EDB2A020ECC
:10AAD00001E3DB2ABBD7070EDB5001E109D1080EE9
:10AAE000DB50110FEA6A000FE96E070EEA22EF5001
:10AAF000E66ED950030FE96EDACFEAFFE552E75070
:10AB0000EE6EED6A030EDBCF00F0040EDBCF01F03A
:10AB100000C001F0006A050E00C0DBFF060E01C098
:10AB2000DBFF080EDB50100FEA6A000FE96E070E1C
:10AB3000EA22EF50E66ED950030FE96EDACFEAFF52
:10AB4000E552E750EE6EED6A050EDBCF00F0060E23
:10AB5000DBCF01F0D950030FE96EDACFEAFF0050E6
:10AB6000EE260150ED22080EDB50F50FE00BE83A1F
:10AB7000E842E66ED9500A0FE96EDACFEAFFE552F5
:10AB8000E750EE6EED6A0A0EDBCF04F00B0EDBCF62
:10AB900005F0050ED89004360536E806FBE11E0EDA
:10ABA0000426000E052204C0E6FF05C0E6FF48ECBF
:10ABB00043F0E552E552F3CF00F0F4CF01F0026A22
:10ABC000036A0C0E00C0DBFF0D0E01C0DBFF0E0E92
:10ABD00002C0DBFF0F0E03C0DBFFD9500C0FE96E84
:10ABE000DACFEAFF040EE76ED890000EEF36010EC2
:10ABF000EB36020EEB36030EEB36E706F5E1D950E5
:10AC00000C0FE96EDACFEAFF040EE76ED890000E63
:10AC1000EF36010EEB36020EEB36030EEB36E7068F
:10AC2000F5E1D9500C0FE96EDACFEAFF040EE76EBA
:10AC3000D890000EEF36010EEB36020EEB36030E07
:10AC4000EB36E706F5E1D9500C0FE96EDACFEAFFF3
:10AC5000040EE76ED890000EEF36010EEB36020EB2
:10AC6000EB36030EEB36E706F5E10A0EDBCF00F01C
:10AC70000B0EDBCF01F0050ED89000360136E8064A
:10AC8000FBE11C0E0026000E012200C0E6FF01C001
:10AC9000E6FF48EC43F0E552E552100EF3CFDBFF40
:10ACA000110EF4CFDBFF100EDBCF04F0110EDBCF63
:10ACB00005F0066A076AD9500C0FE96EDACFEAFF91
:10ACC000EE500424006EEE500520016EEE5006207A
:10ACD000026EEE500720036E0C0E00C0DBFF0D0E5F
:10ACE00001C0DBFF0E0E02C0DBFF0F0E03C0DBFF57
:10ACF00009D1080EDB50110FEA6A000FE96E060E4B
:10AD0000EA22EF50E66ED950030FE96EDACFEAFF80
:10AD1000E552E750EE6EED6A030EDBCF00F0040E55
:10AD2000DBCF01F000C001F0006A050E00C0DBFFC0
:10AD3000060E01C0DBFF080EDB50100FEA6A000FA1
:10AD4000E96E060EEA22EF50E66ED950030FE96E67
:10AD5000DACFEAFFE552E750EE6EED6A050EDBCF83
:10AD600000F0060EDBCF01F0D950030FE96EDACF09
:10AD7000EAFF0050EE260150ED22080EDB50F60FE0
:10AD8000E00BE83AE842E66ED9500A0FE96EDACFF6
:10AD9000EAFFE552E750EE6EED6A0A0EDBCF04F0F3
:10ADA0000B0EDBCF05F0050ED89004360536E8060D
:10ADB000FBE11E0E0426000E052204C0E6FF05C0BE
:10ADC000E6FF48EC43F0E552E552F3CF00F0F4CF54
:10ADD00001F0026A036A0C0E00C0DBFF0D0E01C019
:10ADE000DBFF0E0E02C0DBFF0F0E03C0DBFFD950EE
:10ADF0000C0FE96EDACFEAFF040EE76ED890000E72
:10AE0000EF36010EEB36020EEB36030EEB36E7069D
:10AE1000F5E1D9500C0FE96EDACFEAFF040EE76EC8
:10AE2000D890000EEF36010EEB36020EEB36030E15
:10AE3000EB36E706F5E1D9500C0FE96EDACFEAFF01
:10AE4000040EE76ED890000EEF36010EEB36020EC0
:10AE5000EB36030EEB36E706F5E1D9500C0FE96E41
:10AE6000DACFEAFF040EE76ED890000EEF36010E3F
:10AE7000EB36020EEB36030EEB36E706F5E10A0E73
:10AE8000DBCF00F00B0EDBCF01F0050ED8900036C3
:10AE90000136E806FBE11C0E0026000E012200C070
:10AEA000E6FF01C0E6FF48EC43F0E552E552100E24
:10AEB000F3CFDBFF110EF4CFDBFF100EDBCF04F07E
:10AEC000110EDBCF05F0066A076AD9500C0FE96E48
:10AED000DACFEAFFEE500424006EEE500520016E3A
:10AEE000EE500620026EEE500720036E0C0E00C0DE
:10AEF000DBFF0D0E01C0DBFF0E0E02C0DBFF0F0EED
:10AF000003C0DBFFD950030FE96EDACFEAFF000E72
:10AF1000D880EE54000EED5401E301D1030EDBCFD7
:10AF20000FF0040EDBCF10F0140E0FC0DBFF150E78
:10AF300010C0DBFF120EDB6A130EDB6A030EDBCFE1
:10AF40000FF0040EDBCF10F01C0E0FC0DBFF1D0E48
:10AF500010C0DBFFD9501C0FE96EDACFEAFF000EFC
:10AF6000D880EE54000EED5434E2140EDBCFE6FF31
:10AF7000150EDBCFE6FF1AEC3FF0E552E5521C0E52
:10AF8000F3CFDBFF1D0EF4CFDBFFD9501C0FE96EB2
:10AF9000DACFEAFF000ED880EE54000EED5418E22E
:10AFA0001C0EDBCF0FF01D0EDBCF10F0120E0FC00A
:10AFB000DBFF130E10C0DBFF1C0EDBCF0FF01D0EEE
:10AFC000DBCF10F0140E0FC0DBFF150E10C0DBFF3F
:10AFD000C1D70E01B251046E056A140EDBCF02F028
:10AFE000150EDBCF03F0020E025E000E035A02C004
:10AFF0000FF003C010F004C014F005C015F02DECE4
:10B0000026F00D500E01AE25006E0E50AF21016EE0
:10B01000050E00C0DBFF060E01C0DBFF160EDB6A6B
:10B02000170EDB6A180EDB6A010EF36E1B0EF3CFF0
:10B03000DBFF1B0EDB50000840E2050EDBCFE6FF16
:10B04000060EDBCFE6FF57EC42F0E552E552170E55
:10B05000DB6A180EDB6A1B0EDB50000822E2170EBB
:10B06000DBCF00F0180EDBCF01F0000E005C020E0B
:10B07000015817E2170EDBCFE6FF180EDBCFE6FF15
:10B08000E9EC42F0E552E552E76E1B0EE7CFDBFF3D
:10B09000DB50000805E2170EDB2A180E01E3DB2A5D
:10B0A000DAD71B0EDB50000807E2050EDB2A060E7E
:10B0B00001E3DB2A160EDB2ABCD70E01010E796FE5
:10B0C0007A6B7B6B0A0EDBCF7CFE0B0EDBCF7DFE3B
:10B0D0000C0EDBCF7EFE0D0EDBCF7FFE0E0EDBCF28
:10B0E00080FE0F0EDBCF81FE120EDBCF82FE130E31
:10B0F000DBCF83FE140EDBCF84FE150EDBCF85FE87
:10B10000160EDBCF86FE170EDBCF87FE180EDBCFC9
:10B1100088FEFB0EDBCF8BFEFC0EDBCF8CFE070E1A
:10B12000DB50006E016A00C0F3FF01C0F4FF00D0E5
:10B13000D9CFE1FFE552E7CFD9FF1200D9CFE6FF23
:10B14000E1CFD9FF180EE126DF6A010EDB6A020E9D
:10B15000DB6A030EDB6A040EDB6A010EF36E130E6C
:10B16000F3CFDBFF140EDB6A150EDB6AD950010F3B
:10B17000E96EDACFEAFFEE50ED1020E1200EDF5C41
:10B180001DE2DF500E01016AAC25006EAD510122B7
:10B1900000C0E6FF01C0E6FFC70EE66E010EE66ED8
:10B1A000FFEC4DF0E106E106E106E106DE52F3CFE9
:10B1B000DEFFF4CFDDFFDD52DF2AD8D7DF6A080ECD
:10B1C000DF5C1FE2DF50E76EFD0EDBCFE9FFFE0E16
:10B1D000DBCFEAFFE750E926000EEA22EF50E66EE9
:10B1E000D950050F006EDACF01F0DF500F01EA6B86
:10B1F0000024E96F0150EA23E552E750EF6EDF2AA1
:10B20000DED7090EDF6E0C0EDF5C1FE2DF50E76E4B
:10B21000FD0EDBCFE9FFFE0EDBCFEAFFE750E926AC
:10B22000000EEA22EF50E66ED950050F006EDACF1D
:10B2300001F0DF040F01EA6B0024E96F0150EA23FB
:10B24000E552E750EF6EDF2ADED7010EDBCFE6FFD7
:10B25000020EDBCFE6FFD950050FE66EDACFE6FF30
:10B26000FFEC4DF0E106E106E106E106030EF3CF47
:10B27000DBFF040EF4CFDBFF0E01B251046E056A52
:10B28000010EDBCF0FF0020EDBCF10F0AE510F5CE2
:10B29000026EAF511058036E02C00FF003C010F0E1
:10B2A00004C014F005C015F0B1EC21F00FC000F09F
:10B2B00010C001F0020E0026000E0122110E00C087
:10B2C000DBFF120E01C0DBFFD950130FE96EDACF9E
:10B2D000EAFF000ED880EE54000EED5401E388D052
:10B2E000D950030FE96EDACFEAFFEE50ED1001E01E
:10B2F0007FD0110EDBCFE6FF120EDBCFE6FF1AEC9C
:10B300003FF0E552E552130EF3CFDBFF140EF4CFFE
:10B31000DBFFD950130FE96EDACFEAFF000ED880B9
:10B32000EE54000EED5463E20E01B251046E056A54
:10B33000130EDBCF02F0140EDBCF03F0020E025E21
:10B34000000E035A02C00FF003C010F004C014F046
:10B3500005C015F02DEC26F00D500E01AE25006E47
:10B360000E50AF21016E010E00C0DBFF020E01C0C6
:10B37000DBFF150EDB6A0E01B251F36E150EDBCF4B
:10B38000F4FFF350F45C27E2D950030FE96EDACFF3
:10B39000EAFFEE50ED101FE1010EDBCFE6FF020EDB
:10B3A000DBCFE6FFD950050FE66EDACFE6FFFFEC04
:10B3B0004DF0E106E106E106E106030EF3CFDBFF07
:10B3C000040EF4CFDBFF010EDB2A020E01E3DB2AC1
:10B3D000150EDB2AD0D7130EDBCF0FF0140EDBCF08
:10B3E00010F0110E0FC0DBFF120E10C0DBFF6CD788
:10B3F000030EDBCF00F0040EDBCF01F00E01005096
:10B40000AE5D0150AF5923E2010EDBCFE6FF020E25
:10B41000DBCFE6FFD950050FE66EDACFE6FFB1ECE1
:10B4200054F0E106E106E106E106160EF3CFDBFF7C
:10B43000170EF4CFDBFFD950160FE96EDACFEAFF13
:10B44000EE50ED1002E0FF0E04D0000E02D0000E10
:0EB4500000D0D9CFE1FFE552E7CFD9FF1200BF
:00000001FF
